:0300000002655244
:10655200758E1190000078FF79FFE4F0A3D9FBD883
:0D656200F778FFE4F6D8FD75816F0265AA99
:106886004401D240490FDB4401CE40C90FDB44012D
:05689600CA3C8EFA353A
:0646E4009001B2121F5EFE
:1046EA009001B6E0FCA3E0FDA3E0FEA3E0FFEF2407
:1046FA0069FFEE3474FEED34FFFDEC34FFFCEC127E
:10470A001AC87BDF7A927986783D1218A49001BA8A
:10471A00121F5E7B007A0079C078419001BAE0FCF2
:10472A00A3E0FDA3E0FEA3E0FF1219AD125D4A7BF0
:10473A00007A0079C078411218A4C004C005C006E6
:10474A00C0077F977E7E7DD57C409001BAE0F8A3B2
:10475A00E0F9A3E0FAA3E0FB1217B3D003D002D02A
:10476A0001D0001217AFC004C005C006C0077F926F
:10477A007E867DC07C419001B2E0F8A3E0F9A3E017
:10478A00FAA3E0FB1218A4A804A905AA06AB07D04D
:10479A0007D006D005D0041217B39001C2121F5ECB
:1047AA009001B6E0FCA3E0FDA3E0FEA3E0FFEF2446
:1047BA0069FFEE3474FEED34FFFDEC34FFFCEC12BD
:1047CA001AC89001B2E0F8A3E0F9A3E0FAA3E0FB6B
:1047DA001217B37B307AE67958783D1218A4A804E8
:1047EA00A905AA06AB077F817E0E7DBA7C43121704
:1047FA00AF9001CAE0F8A3E0F9A3E0FAA3E0FB1244
:10480A0018A49001BE121F5E9001CEE0FCA3E0FD49
:10481A00A3E0FEA3E0FF9001BEE0F8A3E0F9A3E065
:10482A00FAA3E0FB121A4A602940279001BEE0FC75
:10483A00A3E0FDA3E0FEA3E0FF9001CEE0F8A3E031
:10484A00F9A3E0FAA3E0FB1217AF9001BE121F5EB4
:10485A0080B69001CEE0FCA3E0FDA3E0FEA3E0FF5A
:10486A00121AB79001BEE0F8A3E0F9A3E0FAA3E0B8
:10487A00FB121A4A50279001BEE0FCA3E0FDA3E018
:10488A00FEA3E0FF9001CEE0F8A3E0F9A3E0FAA3CB
:10489A00E0FB1217B39001BE121F5E80B57F007E47
:1048AA00007D007C009001BEE0F8A3E0F9A3E0FAE5
:1048BA00A3E0FB121A4A604840469001D2E0FCA3EA
:1048CA00E0FDA3E0FEA3E0FF9001BEE0F8A3E0F95B
:1048DA00A3E0FAA3E0FB121A4A50259001BEE0FCBD
:1048EA00A3E0FDA3E0FEA3E0FF9001CEE0F8A3E081
:1048FA00F9A3E0FAA3E0FB1217AF9001BE121F5E04
:10490A007F007E007D007C009001BEE0F8A3E0F904
:10491A00A3E0FAA3E0FB121A4A504B9001D2E0FC42
:10492A00A3E0FDA3E0FEA3E0FF121AB79001BEE0E8
:10493A00F8A3E0F9A3E0FAA3E0FB121A4A602740C1
:10494A00259001BEE0FCA3E0FDA3E0FEA3E0FF90FA
:10495A0001CEE0F8A3E0F9A3E0FAA3E0FB1217B353
:10496A009001BE121F5E9001BEE0FCA3E0FDA3E031
:10497A00FEA3E0FF1254B47B247A0B79987839129B
:10498A0018A49001C2E0F8A3E0F9A3E0FAA3E0FBBF
:10499A001217B39001C6121F5E7B007A0079C078A5
:1049AA00419001C6E0FCA3E0FDA3E0FEA3E0FF12F4
:1049BA0019AD125D4A7B007A0079C078411218A4B9
:1049CA00A804A905AA06AB079001C6E0FCA3E0FD6E
:0949DA00A3E0FEA3E0FF1217AFF9
:0149E30022B1
:106844009001DD121F5E9001DDE0FCA3E0FDA3E0FA
:10685400FEA3E0FF125D4AA804A905AA06AB0790AF
:1068640001DDE0FCA3E0FDA3E0FEA3E0FF1217AF0F
:106874009001CEE0F8A3E0F9A3E0FAA3E0FB12183C
:02688400A4224C
:060C7D00900142121F5E0F
:100C8300900142E0FCA3E0FDA3E0FEA3E0FFEF241C
:100C930013FFEE342DFEED34FFFDEC34FFFCEC12BC
:100CA3001AC8900146E0F8A3E0F9A3E0FAA3E0FB39
:100CB3001217B390014A121F5E7F8D7EA67D147CAE
:100CC3003D90014AE0F8A3E0F9A3E0FAA3E0FB12A8
:100CD30018A47B807AF279BF783E1217B312684466
:100CE30090014E121F5E7F477E857D167C3D9001ED
:100CF3004AE0F8A3E0F9A3E0FAA3E0FB1218A47B0F
:100D0300937AA77984783E1217B3126844900152FC
:100D1300121F5E7F217EB47D0A7C3D90014AE0F87C
:100D2300A3E0F9A3E0FAA3E0FB1218A47BFF7ACDBA
:100D33007953783F1217B3126844900156121F5E1D
:100D43007F4D7E6C7D337C3B90014AE0F8A3E0F954
:100D5300A3E0FAA3E0FB1218A47B817A3D797E78A5
:100D63003F1217B312684490015A121F5E7F007E30
:100D7300007D007C40900156E0F8A3E0F9A3E0FA7F
:100D8300A3E0FB1218A4A804A905AA06AB079001C7
:100D93004EE0FCA3E0FDA3E0FEA3E0FF1217AF12B9
:100DA300549E7BF37A767914783F1218A4C004C05A
:100DB30005C006C00790014EE0FCA3E0FDA3E0FEE2
:100DC300A3E0FF12549E7BE87AC179517840121850
:100DD300A4A804A905AA06AB077FB17E737D717C25
:100DE300421217AFD003D002D001D0001217AFC008
:100DF30004C005C006C0077F007E007D007C4090D4
:100E03000156E0F8A3E0F9A3E0FAA3E0FB1218A46B
:100E130012549E7B0C7A5979ED783E1218A4A804DB
:100E2300A905AA06AB07D007D006D005D004121730
:100E3300AF90015E121F5E7F007E007D007C4090BC
:100E43000156E0F8A3E0F9A3E0FAA3E0FB1218A42B
:100E5300C004C005C006C0077F007E007D007C4043
:100E630090014EE0F8A3E0F9A3E0FAA3E0FB121827
:100E7300A4D003D002D001D0001217AF12549E7B2E
:100E8300767A4F791E783D1218A4C004C005C006B7
:100E9300C0077F007E007D007C4090014EE0F8A3F8
:100EA300E0F9A3E0FAA3E0FB1218A412549E7B9C82
:100EB3007A5A79B6783D1218A4A804A905AA06ABF4
:100EC3000790015EE0FCA3E0FDA3E0FEA3E0FF12B8
:100ED30017AFA804A905AA06AB07D007D006D0050B
:100EE300D0041217B3C004C005C006C0077F007E3C
:100EF300007D007C40900156E0F8A3E0F9A3E0FAFE
:100F0300A3E0FB1218A490015AE0F8A3E0F9A3E0D0
:100F1300FAA3E0FB1217AF12549E7B687A9679040A
:100F2300783D1218A4A804A905AA06AB07D007D0D8
:100F330006D005D0041217AF90015E121F5E7F002A
:100F43007E007D007C40900156E0F8A3E0F9A3E029
:100F5300FAA3E0FB1218A4A804A905AA06AB0790FC
:100F6300014EE0FCA3E0FDA3E0FEA3E0FF1217AFF8
:100F730090015AE0F8A3E0F9A3E0FAA3E0FB12170B
:100F8300B312549E7BD87A2A79C1783C1218A4C034
:100F930004C005C006C0077F007E007D007C409032
:100FA3000156E0F8A3E0F9A3E0FAA3E0FB1218A4CA
:100FB300A804A905AA06AB0790014EE0FCA3E0FD37
:100FC300A3E0FEA3E0FF1217AF12549E7B727A33A5
:100FD30079DC783C1218A4A804A905AA06AB0790EB
:100FE300015EE0FCA3E0FDA3E0FEA3E0FF1217AF68
:100FF300D003D002D001D0001217AFC004C005C087
:1010030006C00790015AE0F8A3E0F9A3E0FAA3E0D1
:10101300FB90014EE0FCA3E0FDA3E0FEA3E0FF1282
:1010230017AF12549E7B307A4C79A6783C1218A4E1
:10103300A804A905AA06AB07D007D006D005D0049B
:101043001217AF90015E121F5E900156E0FCA3E001
:10105300FDA3E0FEA3E0FF12549E7B0B7AD2798CB2
:10106300783C1218A490015EE0F8A3E0F9A3E0FA3B
:10107300A3E0FB1217B3C004C005C006C00790016C
:101083005AE0FCA3E0FDA3E0FEA3E0FF90014EE0E5
:10109300F8A3E0F9A3E0FAA3E0FB1217B312549EFE
:1010A3007B697AE37988783C1218A4A804A905AA75
:1010B30006AB07D007D006D005D0041217B39001B2
:1010C3005E121F5E7F007E007D007C40900152E037
:1010D300F8A3E0F9A3E0FAA3E0FB1218A4A804A97B
:1010E30005AA06AB0790014EE0FCA3E0FDA3E0FEDA
:1010F300A3E0FF1217AF12549E7BF97A4E794C7816
:101103003C1218A4C004C005C006C00790015AE0F1
:10111300FCA3E0FDA3E0FEA3E0FF12549E7BCD7A87
:10112300AF79E6783B1218A4A804A905AA06AB0771
:10113300D007D006D005D0041217B3C004C005C031
:1011430006C0077F007E007D007C40900156E0F8DA
:10115300A3E0F9A3E0FAA3E0FB1218A490015AE07C
:10116300F8A3E0F9A3E0FAA3E0FB1217B312549E2D
:101173007BBC7A5779AD783B1218A4A804A905AAB9
:1011830006AB07D007D006D005D0041217B3C004AE
:10119300C005C006C0077F007E007D807C409001B3
:1011A30056E0F8A3E0F9A3E0FAA3E0FB1218A4A821
:1011B30004A905AA06AB0790014EE0FCA3E0FDA33A
:1011C300E0FEA3E0FF1217AF12549E7B4E7AB47970
:1011D300AB783B1218A4A804A905AA06AB07D0074D
:1011E300D006D005D0041217AF900162121F5E7FA4
:1011F300007E007D007C40900156E0F8A3E0F9A357
:10120300E0FAA3E0FB1218A4A804A905AA06AB07F9
:1012130090014EE0FCA3E0FDA3E0FEA3E0FF121764
:10122300AF90015AE0F8A3E0F9A3E0FAA3E0FB12C0
:1012330017AF12549E7BA97A6A7982783B1218A45D
:10124300900162E0F8A3E0F9A3E0FAA3E0FB121730
:10125300B3C004C005C006C0077F007E007D407C8C
:101263004090014EE0F8A3E0F9A3E0FAA3E0FB12FB
:1012730018A412549E7B9C7ADC796F783B1218A4D5
:10128300A804A905AA06AB07D007D006D005D00449
:101293001217AFC004C005C006C0077F007E007DE3
:1012A300807C40900156E0F8A3E0F9A3E0FAA3E0C4
:1012B300FB1218A4C004C005C006C0077F007E004F
:1012C3007D007C4090014EE0F8A3E0F9A3E0FAA38F
:1012D300E0FB1218A4D003D002D001D0001217AF44
:1012E30012549E7BCA7A547941783B1218A4A804FD
:1012F300A905AA06AB07D007D006D005D00412175C
:10130300AF900162121F5E7F007E007D007C4090E3
:101313000156E0F8A3E0F9A3E0FAA3E0FB1218A456
:10132300C004C005C006C0077F007E007D407C402E
:1013330090014EE0F8A3E0F9A3E0FAA3E0FB121852
:10134300A4D003D002D001D0001217AF12549E7B59
:10135300457A2F7923783B1218A4C004C005C00630
:10136300C00790015AE0FCA3E0FDA3E0FEA3E0FF69
:10137300900156E0F8A3E0F9A3E0FAA3E0FB12170B
:10138300B312549E7B147A5C792C783B1218A4A870
:1013930004A905AA06AB07900162E0FCA3E0FDA344
:1013A300E0FEA3E0FF1217AFA804A905AA06AB0746
:1013B300D007D006D005D0041217B3C004C005C0AF
:1013C30006C0077F007E007D007C40900156E0F858
:1013D300A3E0F9A3E0FAA3E0FB1218A490014EE006
:1013E300F8A3E0F9A3E0FAA3E0FB1217B390015AC4
:1013F300E0F8A3E0F9A3E0FAA3E0FB1217AF12545D
:101403009E7BA67AD57910783B1218A4A804A90567
:10141300AA06AB07D007D006D005D0041217AFC079
:1014230004C005C006C0077F007E007D007C40909D
:101433000156E0F8A3E0F9A3E0FAA3E0FB1218A435
:10144300C004C005C006C0077F007E007D007C404D
:10145300900152E0F8A3E0F9A3E0FAA3E0FB12182D
:10146300A4D003D002D001D0001217AF12549E7B38
:10147300B37A7B79F2783A1218A4A804A905AA06CC
:10148300AB07D007D006D005D0041217B390016282
:10149300121F5E7F007E007D007C40900152E0F8C9
:1014A300A3E0F9A3E0FAA3E0FB1218A490014EE035
:1014B300F8A3E0F9A3E0FAA3E0FB1217B3C004C05A
:1014C30005C006C0077F007E007D007C409001566A
:1014D300E0F8A3E0F9A3E0FAA3E0FB1218A4A80440
:1014E300A905AA06AB07D007D006D005D00412176A
:1014F300AF12549E7B047AAD79C0783A1218A4C017
:1015030004C005C006C0077F007E007D007C4090BC
:10151300015AE0F8A3E0F9A3E0FAA3E0FB1218A450
:10152300C004C005C006C0077F007E007D007C406C
:10153300900156E0F8A3E0F9A3E0FAA3E0FB121848
:10154300A4D003D002D001D0001217AF12549E7B57
:10155300A37A0679D378BA1218A4A804A905AA060F
:10156300AB07D007D006D005D0041217B3C004C010
:1015730005C006C0077F007E007D807C4090015639
:10158300E0F8A3E0F9A3E0FAA3E0FB1218A41254D5
:101593009E7B4B7A1F79BA783A1218A4A804A9053E
:1015A300AA06AB07D007D006D005D0041217AFC0E8
:1015B30004C005C006C0077F007E007D007C40900C
:1015C3000156E0F8A3E0F9A3E0FAA3E0FB1218A4A4
:1015D300C004C005C006C0077F007E007D007C40BC
:1015E30090014EE0F8A3E0F9A3E0FAA3E0FB1218A0
:1015F300A4D003D002D001D0001217AF90015AE05B
:10160300F8A3E0F9A3E0FAA3E0FB1217B312549E88
:101613007BA97A3079B6783A1218A4A804A905AA46
:1016230006AB07D007D006D005D0041217B390013C
:1016330066121F5E7F007E007D807C40900156E035
:10164300F8A3E0F9A3E0FAA3E0FB1218A4A804A905
:1016530005AA06AB0790014EE0FCA3E0FDA3E0FE64
:10166300A3E0FF1217AF90015AE0F8A3E0F9A3E05B
:10167300FAA3E0FB1217B312549E7B3B7AAA799A22
:10168300783A1218A4A804A905AA06AB0790016624
:10169300E0FCA3E0FDA3E0FEA3E0FF1217AFC0044C
:1016A300C005C006C0077F007E007D007C4090011E
:1016B30056E0F8A3E0F9A3E0FAA3E0FB1218A4C0F4
:1016C30004C005C006C0077F007E007D007C4090FB
:1016D300014EE0F8A3E0F9A3E0FAA3E0FB1218A49B
:1016E300A804A905AA06AB07D007D006D005D004E5
:1016F3001217B312549E7B247A0B7998783A1218F6
:10170300A4A804A905AA06AB07D007D006D005D024
:10171300041217AFC004C005C006C0077F007E00D7
:101723007D007C4090014EE0F8A3E0F9A3E0FAA32A
:10173300E0FB1218A490015AE0F8A3E0F9A3E0FA41
:10174300A3E0FB1217AF12549E7BE07A2D799078B9
:101753003A1218A4A804A905AA06AB07D007D00615
:10176300D005D0041217AF900166121F5E9001627C
:10177300E0FCA3E0FDA3E0FEA3E0FF90015EE0F840
:10178300A3E0F9A3E0FAA3E0FB1217B3900166E02C
:10179300F8A3E0F9A3E0FAA3E0FB1217B37B487ABE
:0817A3005179C778451218A422
:0117AB00221B
:0B29D500900108EBF0A3EAF0A3E9F08A
:1029E00090010EE0FCA3E0FDA3E0FEA3E0FFEC12EB
:1029F0001AC87B007A81798878C61217B3900112C1
:102A0000E0F8A3E0F9A3E0FAA3E0FB1217B390010A
:102A100016121F5E7F0A7EEB7D157C3D900116E04D
:102A2000F8A3E0F9A3E0FAA3E0FB1218A47B7F7AF5
:102A30004F7940783F1217B312684490011A121F61
:102A40005E7F8C7EA67D147C3D900116E0F8A3E0AD
:102A5000F9A3E0FAA3E0FB1218A47B367A9079522E
:102A6000783F1217B312684490011E121F5E7F4D0B
:102A70007E6C7D337C3B900116E0F8A3E0F9A3E087
:102A8000FAA3E0FB1218A47B857AEA797E783F12DC
:102A900017B3126844900122121F5E7F217EB47D1D
:102AA0000A7C3D900116E0F8A3E0F9A3E0FAA3E068
:102AB000FB1218A47BD37A697979783F1217B31285
:102AC0006844900126121F5E7F477E857D167C3DFF
:102AD000900116E0F8A3E0F9A3E0FAA3E0FB1218D6
:102AE000A47B9F7A027900783D1217B31268449054
:102AF000012A121F5E7F007E007D007C409001262F
:102B0000E0F8A3E0F9A3E0FAA3E0FB1218A4125442
:102B1000B47BB07A727928783F1218A4C004C0053B
:102B2000C006C00790011EE0FCA3E0FDA3E0FEA3E9
:102B3000E0FF1254B47B7D7A3F79C978401218A423
:102B4000A804A905AA06AB07D007D006D005D00473
:102B50001217B3C004C005C006C0077F007E007D09
:102B6000007C40900126E0F8A3E0F9A3E0FAA3E09E
:102B7000FB1218A4A804A905AA06AB0790011EE041
:102B8000FCA3E0FDA3E0FEA3E0FF1217AF1254B4D4
:102B90007B6F7A1279A3783F1218A4A804A905AA1A
:102BA00006AB07D007D006D005D0041217AFC0047B
:102BB000C005C006C007900122E0FCA3E0FDA3E031
:102BC000FEA3E0FF1254B47BC97A76793E783E12B8
:102BD00018A4A804A905AA06AB07D007D006D005FB
:102BE000D0041217AF9001CAE0F8A3E0F9A3E0FA0D
:102BF000A3E0FB1218A490011AE0F8A3E0F9A3E007
:102C0000FAA3E0FB1217B390012E121F5E90012E63
:102C1000E0FCA3E0FDA3E0FEA3E0FFC004C005C00C
:102C200006C0077F007E007D007C4090012AE0F80E
:102C3000A3E0F9A3E0FAA3E0FB1218A41254B47BBA
:102C4000D57A7879E9783D1218A4C004C005C00689
:102C5000C0077F007E007D007C4090011EE0F8A34D
:102C6000E0F9A3E0FAA3E0FB1218A41254B47BD15C
:102C70007A22795B783E1218A4D003D002D001D01A
:102C8000001217AFC004C005C006C0077F007E0059
:102C90007D007C40900126E0F8A3E0F9A3E0FAA3D0
:102CA000E0FB1218A4C004C005C006C0077F007E68
:102CB000007D007C4090011EE0F8A3E0F9A3E0FA5B
:102CC000A3E0FB1218A4D003D002D001D000121749
:102CD000AF1254B47BFC7AA97971783D1218A4A87C
:102CE00004A905AA06AB07D007D006D005D0041268
:102CF00017AFC004C005C006C0077F007E007D007E
:102D00007C40900126E0F8A3E0F9A3E0FAA3E0FB01
:102D10001218A4C004C005C006C007900122E0FC40
:102D2000A3E0FDA3E0FEA3E0FF90011EE0F8A3E016
:102D3000F9A3E0FAA3E0FB1217B3D003D002D0014D
:102D4000D0001217AF1254B47BD57A787969783DE8
:102D50001218A4A804A905AA06AB07D007D006D06C
:102D600005D0041217AF9001CAE0F8A3E0F9A3E080
:102D7000FAA3E0FB1218A4A804A905AA06AB07D081
:102D800007D006D005D0041217B390012E121F5E93
:102D90007F007E007D007C40900126E0F8A3E0F9F2
:102DA000A3E0FAA3E0FB1218A41254B47BE37AC7A1
:102DB0007928783F1218A4C004C005C006C0079047
:102DC000011EE0FCA3E0FDA3E0FEA3E0FF1254B46B
:102DD0007B9E7A5E79C778401218A4A804A905AA38
:102DE00006AB07D007D006D005D0041217B3C00435
:102DF000C005C006C0077F007E007D007C409001BA
:102E000026E0F8A3E0F9A3E0FAA3E0FB1218A4A8D7
:102E100004A905AA06AB0790011EE0FCA3E0FDA3F0
:102E2000E0FEA3E0FF1217AF1254B47BE57AD0792D
:102E3000A2783F1218A4A804A905AA06AB07D007D8
:102E4000D006D005D0041217AF9001CAE0F8A3E075
:102E5000F9A3E0FAA3E0FB1218A490012AE0F8A37A
:102E6000E0F9A3E0FAA3E0FB1217B3900132121FBE
:102E70005E7F007E007D007C40900126E0F8A3E0AC
:102E8000F9A3E0FAA3E0FB1218A4A804A905AA0676
:102E9000AB0790012AE0FCA3E0FDA3E0FEA3E0FF66
:102EA0001217AF1254B47B067A817915783E121846
:102EB000A4C004C005C006C007900132E0FCA3E036
:102EC000FDA3E0FEA3E0FF1254B47BA67A9B79A495
:102ED00078401218A4D003D002D001D0001217AF4E
:102EE0009001CAE0F8A3E0F9A3E0FAA3E0FB12180E
:102EF000A4900136121F5E90012EE0FCA3E0FDA31A
:102F0000E0FEA3E0FF1254B4C004C005C006C00731
:102F1000900136E0FCA3E0FDA3E0FEA3E0FF125425
:102F20009EA804A905AA06AB07D007D006D005D0F5
:102F3000041218A47B327AAF79CB783E1218A4C061
:102F400004C005C006C007900136E0FCA3E0FDA365
:102F5000E0FEA3E0FF1254B47BDB7ADE796A783FAF
:102F60001218A4A804A905AA06AB07D007D006D05A
:102F700005D0041217B390010BE0FBA3E0FAA3E025
:102F8000F9121EEC90010BE0FBA3E0FAA3E0F912AA
:102F90001ECC90010BE0FBA3E0FAA3E0F9121F3E68
:102FA0001218A4A804A905AA06AB077F007E007D1D
:102FB000807C3F1217AF1263629000D0121F5E90A8
:102FC000010BE0FBA3E0FAA3E0F9121ECC1265EFBF
:102FD00090010BE0FBA3E0FAA3E0F9121EEC9001D4
:102FE0002EE0FCA3E0FDA3E0FEA3E0FF12549EC090
:102FF00004C005C006C007900136E0FCA3E0FDA3B5
:10300000E0FEA3E0FF12549EA804A905AA06AB07A0
:10301000D007D006D005D0041218A4C004C005C043
:1030200006C00790010BE0FBA3E0FAA3E0F9121E33
:10303000CC12549EA804A905AA06AB07D007D00657
:10304000D005D0041219AD90013A121F5E90012EE6
:10305000E0FCA3E0FDA3E0FEA3E0FF1254B4C00433
:10306000C005C006C007900136E0FCA3E0FDA3E068
:10307000FEA3E0FF12549EA804A905AA06AB07D040
:1030800007D006D005D0041218A47BDB7ADE796A5B
:10309000783F1218A4C004C005C006C007900136CE
:1030A000E0FCA3E0FDA3E0FEA3E0FF1254B47B32FA
:1030B0007AAF79CB783E1218A4A804A905AA06AB6A
:1030C00007D007D006D005D0041217AFC004C00542
:1030D000C006C00790010BE0FBA3E0FAA3E0F912E1
:1030E0001ECC12549EA804A905AA06AB07D007D08F
:1030F00006D005D0041219AD90013E121F5E90015A
:103100003EE0FCA3E0FDA3E0FEA3E0FFC004C00599
:10311000C006C00790013AE0FCA3E0FDA3E0FEA3D7
:10312000E0FF9000D0121F5ED007D006D005D0047B
:103130001265EF900108E0FBA3E0FAA3E0F9121E8C
:10314000EC900108E0FBA3E0FAA3E0F9121ECC7BAF
:10315000007A0079007800121A4A6030402E9001FF
:1031600008E0FBA3E0FAA3E0F9C003C002C001122B
:103170001ECC9001CEE0F8A3E0F9A3E0FAA3E0FBB7
:103180001217B3D001D002D003121EEC900108E058
:10319000FBA3E0FAA3E0F9121ECC9001CEE0F8A365
:1031A000E0F9A3E0FAA3E0FB121A4A502E900108BE
:1031B000E0FBA3E0FAA3E0F9C003C002C001121EC5
:1031C000CC9001CEE0F8A3E0F9A3E0FAA3E0FB1273
:0B31D00017AFD001D002D003121EEC9C
:0131DB0022D1
:0B3FC100900190EBF0A3EAF0A3E9F000
:103FCC00900196E0FCA3E0FDA3E0FEA3E0FFEC1261
:103FDC001AC87B007A81798878C61217B390019A37
:103FEC00E0F8A3E0F9A3E0FAA3E0FB1217B37B001F
:103FFC007AAD790E78471219AD90019E121F5E7F33
:10400C00A67EFE7DC77C4290019EE0F8A3E0F9A35A
:10401C00E0FAA3E0FB1218A47B917AEA797E783F50
:10402C001217B31268449001A2121F5E7F117E23F7
:10403C007D5F7C3790019EE0F8A3E0F9A3E0FAA342
:10404C00E0FB1218A4A804A905AA06AB077F507EB2
:10405C00AC7DAE7C3B1217AF126844C004C005C0E7
:10406C0006C0079001A2E0FCA3E0FDA3E0FEA3E0E4
:10407C00FF1254B4A804A905AA06AB07D007D006B2
:10408C00D005D0041218A4C004C005C006C0077F18
:10409C00187E017DC87C4290019EE0F8A3E0F9A354
:1040AC00E0FAA3E0FB1218A47B327AE47946783F5D
:1040BC001217B3126844A804A905AA06AB07D007C7
:1040CC00D006D005D0041217B3C004C005C006C07A
:1040DC00077F007E007D007C409001A2E0F8A3E009
:1040EC00F9A3E0FAA3E0FB1218A41254B47B0C7AE7
:1040FC0034796978381218A4A804A905AA06AB0764
:10410C00D007D006D005D0041217B39001A6121F09
:10411C005E7F147E6A7D177C3890019EE0F8A3E0E8
:10412C00F9A3E0FAA3E0FB1218A4A804A905AA06B7
:10413C00AB077F6D7E6A7D857C3D1217AF1268449C
:10414C009001AA121F5E9001A6E0FCA3E0FDA3E083
:10415C00FEA3E0FF1254F0C004C005C006C00790D7
:10416C0001AAE0FCA3E0FDA3E0FEA3E0FF12549E35
:10417C00A804A905AA06AB07D007D006D005D00421
:10418C001218A41255FE900190E0FBA3E0FAA3E0F4
:10419C00F9121EEC9001CEE0F8A3E0F9A3E0FAA32B
:1041AC00E0FB9001A6E0FCA3E0FDA3E0FEA3E0FF92
:1041BC001219AD125D4A9001CEE0F8A3E0F9A3E02C
:1041CC00FAA3E0FB1218A4A804A905AA06AB079051
:1041DC0001A6E0FCA3E0FDA3E0FEA3E0FF1217AFF5
:1041EC009001AE121F5E7F007E007DC07C3F90016F
:1041FC00D2E0F8A3E0F9A3E0FAA3E0FB1218A49034
:10420C0001AEE0F8A3E0F9A3E0FAA3E0FB121A4A2E
:10421C00505A7F007E007D007C3F9001D2E0F8A3D5
:10422C00E0F9A3E0FAA3E0FB1218A49001AEE0F8C9
:10423C00A3E0F9A3E0FAA3E0FB121A4A402E900186
:10424C0090E0FBA3E0FAA3E0F9C003C002C00112A6
:10425C001ECC9001D2E0F8A3E0F9A3E0FAA3E0FBB6
:10426C001217B3D001D002D003121EEC900190E0D3
:10427C00FBA3E0FAA3E0F9C003C002C001121ECCFC
:10428C00C004C005C006C007900190E0FBA3E0FA93
:10429C00A3E0F9121ECC9001CEE0F8A3E0F9A3E064
:1042AC00FAA3E0FB1219AD125D4A9001CEE0F8A31F
:1042BC00E0F9A3E0FAA3E0FB1218A4A804A905AA4C
:1042CC0006AB07D007D006D005D0041217AFD0012B
:1042DC00D002D003121EEC9001A6E0FCA3E0FDA3DB
:1042EC00E0FEA3E0FF1254B4C004C005C006C00732
:1042FC009001AAE0FCA3E0FDA3E0FEA3E0FF1254B2
:10430C00B4A804A905AA06AB07D007D006D005D0DF
:10431C00041218A4900193E0FBA3E0FAA3E0F912B5
:10432C001EEC900193E0FBA3E0FAA3E0F9121ECC83
:10433C00900193E0FBA3E0FAA3E0F9121F3E1218E0
:10434C00A4A804A905AA06AB077F007E007D807C8B
:10435C003F1217AF1263629000D0121F5E90019350
:10436C00E0FBA3E0FAA3E0F9121ECC1265EF90017A
:0C437C0093E0FBA3E0FAA3E0F9121EECB2
:014388002212
:0B31DC0090016AEBF0A3EAF0A3E9F019
:1031E7007F927E0A7D867C3E900170E0F8A3E0F92D
:1031F700A3E0FAA3E0FB1218A4900174E0F8A3E09F
:10320700F9A3E0FAA3E0FB1217AF90017C121F5E4F
:103217007F007E007D007C0090017CE0F8A3E0F950
:10322700A3E0FAA3E0FB121A4A502790017CE0FCC6
:10323700A3E0FDA3E0FEA3E0FF9001CEE0F8A3E04A
:10324700F9A3E0FAA3E0FB1217B390017C121F5E0B
:1032570080489001CEE0FCA3E0FDA3E0FEA3E0FFE1
:1032670090017CE0F8A3E0F9A3E0FAA3E0FB121ACF
:103277004A6027402590017CE0FCA3E0FDA3E0FE27
:10328700A3E0FF9001CEE0F8A3E0F9A3E0FAA3E002
:10329700FB1217AF90017C121F5E90017CE0F8A330
:1032A700E0F9A3E0FAA3E0FB90001EE0FCA3E0FD39
:1032B700A3E0FEA3E0FF1217AF900016121F5E9067
:1032C7000016E0FCA3E0FDA3E0FEA3E0FF12549E7E
:1032D700C004C005C006C00790001AE0FCA3E0FDCB
:1032E700A3E0FEA3E0FF12549EA804A905AA06AB1B
:1032F70007D007D006D005D0041218A4C004C00513
:10330700C006C007900178E0FCA3E0FDA3E0FEA3A0
:10331700E0FF12549EA804A905AA06AB07D007D060
:1033270006D005D0041218A4C004C005C006C00703
:1033370090001AE0FCA3E0FDA3E0FEA3E0FF125417
:10334700B4C004C005C006C007900178E0FCA3E044
:10335700FDA3E0FEA3E0FF1254B4A804A905AA0642
:10336700AB07D007D006D005D0041218A4A804A92B
:1033770005AA06AB07D007D006D005D0041217B3AD
:10338700900180121F5E900180E0FCA3E0FDA3E0A6
:10339700FEA3E0FF900180E0F8A3E0F9A3E0FAA321
:1033A700E0FB1218A4A804A905AA06AB077F007EB4
:1033B700007D807C3F1217AF126362900184121F59
:1033C7005E900180E0FCA3E0FDA3E0FEA3E0FFC068
:1033D70004C005C006C007900184E0FCA3E0FDA37C
:1033E700E0FEA3E0FF9000D0121F5ED007D006D00A
:1033F70005D0041265EF90016DE0FBA3E0FAA3E0AE
:10340700F9121EEC90016DE0FBA3E0FAA3E0F912BC
:103417001ECC12549EC004C005C006C00790016DA3
:10342700E0FBA3E0FAA3E0F9121ECC1254B4D003D8
:10343700D002D001D0001219ADC004C005C006C02B
:103447000790001AE0FCA3E0FDA3E0FEA3E0FF1253
:10345700549EC004C005C006C00790001AE0FCA334
:10346700E0FDA3E0FEA3E0FF1254B4D003D002D0E6
:1034770001D0001219ADA804A905AA06AB07D00709
:10348700D006D005D0041218A4C004C005C006C0D9
:103497000790016DE0FBA3E0FAA3E0F9121ECC123E
:1034A700549EC004C005C006C00790001AE0FCA3E4
:1034B700E0FDA3E0FEA3E0FF12549EA804A905AA1D
:1034C70006AB07D007D006D005D0041218A4C00455
:1034D700C005C006C007900178E0FCA3E0FDA3E0AB
:1034E700FEA3E0FF1254B4D003D002D001D00012E3
:1034F70019ADD003D002D001D0001217AF90018CC4
:10350700121F5E900178E0FCA3E0FDA3E0FEA3E0BC
:10351700FF12549EC004C005C006C00790001AE001
:10352700FCA3E0FDA3E0FEA3E0FF12549EA804A9BC
:1035370005AA06AB07D007D006D005D0041218A4F9
:10354700C004C005C006C007900016E0FCA3E0FD5C
:10355700A3E0FEA3E0FF12549EA804A905AA06ABA8
:1035670007D007D006D005D0041218A4C004C005A0
:10357700C006C007900178E0FCA3E0FDA3E0FEA32E
:10358700E0FF1254B4C004C005C006C00790001A7B
:10359700E0FCA3E0FDA3E0FEA3E0FF1254B4A804FF
:1035A700A905AA06AB07D007D006D005D004121884
:1035B700A4A804A905AA06AB07D007D006D005D052
:1035C700041217B3900188121F5E900178E0FCA3E4
:1035D700E0FDA3E0FEA3E0FF12549EC004C005C0B7
:1035E70006C007900016E0FCA3E0FDA3E0FEA3E001
:1035F700FF1254B4A804A905AA06AB07D007D00642
:10360700D005D0041218A4C004C005C006C0079096
:103617000188E0FCA3E0FDA3E0FEA3E0FF900188A2
:10362700E0F8A3E0F9A3E0FAA3E0FB1218A4A804CA
:10363700A905AA06AB077F007E007D807C3F121795
:10364700AF126362A804A905AA06AB07D007D00684
:10365700D005D0041219AD900188121F5E90018821
:10366700E0FCA3E0FDA3E0FEA3E0FFC004C005C0AB
:1036770006C00790018CE0FCA3E0FDA3E0FEA3E0F9
:10368700FF9000D0121F5ED007D006D005D00412DD
:1036970065EF90016AE0FBA3E0FAA3E0F9121EECE4
:1036A70090016AE0FBA3E0FAA3E0F9121ECC7B00CD
:1036B7007A0079007800121A4A6030402E90016A29
:1036C700E0FBA3E0FAA3E0F9C003C002C001121EA9
:1036D700CC9001CEE0F8A3E0F9A3E0FAA3E0FB1257
:0B36E70017B3D001D002D003121EEC7C
:0136F20022B5
:1062B200323B171C0205006400640001000007A3C2
:1062C20000870384006407080384068205690007C7
:1062D20000020009003B003B0017001C000C006399
:1062E20000C700C70002000A0E0F03840E0F0384CA
:1062F2000E0F07080E0F070800070005000E00002A
:106302000000000000010001000000010001000087
:10631200000000000000000000000000000000007B
:106322000000000000000000000000030000000365
:106332000002000300020003000300020003000247
:10634200000300000003000100030002000300023A
:0C6352000003000300020003000200032F
:06689B00C112C114C1137B
:10671D009000107432F0900011743BF090001274E0
:10672D0017F0900013741CF09000147402F0900098
:10673D00157405F0124CAD756100756200D3E562FC
:10674D00940EE56164809480503CE56225E0FFE5A0
:10675D006133FE74B82FF58274623EF583E493FCC9
:10676D00740193FDE56225E0FFE56133FE74222F90
:10677D00F58274003EF583ECF0A3EDF00562E56261
:0A678D007002056180B7124DB122C1
:103B760090003FE0F55CD3E55C64809482400BC323
:103B8600E55C648094865002C212E5A064FFFFEFF4
:103B96005407F55EE55E6006C29CC2988002D29C20
:103BA600E55E5406FFEF60270560E560D3940A40A2
:103BB6000F755D0AC3E55C64809486500375600AE0
:103BC600E560D39414400E755D64756014800675C7
:103BD6006000755D01AF5CEF3395E0FEEF25E0FF19
:103BE600EE33FE74002FF58274633EF583E493F59D
:103BF6005A740193F55BAF5CEF3395E0FEEF25E079
:103C0600FFEE33FE74D62FF58274623EF583E4939D
:103C1600F558740193F559E55C6403706B900015D3
:103C2600E0FFEF75F004121D86AFF0EF602E9000F6
:103C360014E0FFEF3395E0FEEF25E0FFEE33FE7470
:103C46002A2FF58274633EF583E493FE740193FF95
:103C5600EF2559F559EE3558F558802C900014E0AB
:103C6600FFEF3395E0FEEF25E0FFEE33FE74442FC1
:103C7600F58274633EF583E493FE740193FFEF25AA
:103C860059F559EE3558F558E55EB40110900028FF
:103C9600E0FEA3E0FFEF4E7004055F8003755F0052
:103CA600E55FC394144008755F00A212B39212D365
:103CB600E55E648094815003023F65C3E55C6480E1
:103CC60094864003023D8B124D02E55E64047055F6
:103CD600AF5CEF3395E0FE74102FF58274003EF56D
:103CE60083E0255DF0AF5CEF3395E0FE74102FF5B1
:103CF6008274003EF583E0FFEF3395E0FED3EF9547
:103D060059E5586480F8EE6480984016AF5BAE5C67
:103D1600EEFD3395E0FC74102DF58274003CF583BE
:103D2600EFF0124CADE55E6402705AAF5CEF33956E
:103D3600E0FE74102FF58274003EF583E0FFC3EFBA
:103D4600955DFFEFF0AF5CEF3395E0FE74102FF555
:103D56008274003EF583E0FFEF3395E0FEC3EF95F6
:103D66005BE55A6480F8EE6480985016AF59AE5CF5
:103D7600EEFD3395E0FC74102DF58274003CF5835E
:103D8600EFF0124CADC3E55C648094865003023EAE
:103D9600A774FA255CF55CE55E64047072AF5DEFAE
:103DA600FD7C00AF5CEF3395E0FEEF25E0FFEE33E0
:103DB600FE74222FF58274003EF583EC8DF0121E00
:103DC60048AF5CEF3395E0FEEF25E0FFEE33FE747F
:103DD600222FF58274003EF583E0FEA3E0FFD3EFC9
:103DE6009559E5586480F8EE648098401FAF5CEF03
:103DF6003395E0FEEF25E0FFEE33FE74222FF582C9
:103E060074003EF583E55AF0A3E55BF0124DB1E58B
:103E16005E64026003023EA1AF5CEF3395E0FEEF05
:103E260025E0FFEE33FE74222FF58274003EF58303
:103E3600C083C082E0FEA3E0FFAD5D7C00C3EF9DC2
:103E4600FFEE9CFED082D083EEF0A3EFF0AF5CEFE6
:103E56003395E0FEEF25E0FFEE33FE74222FF58268
:103E660074003EF583E0FEA3E0FFC3EF955BE55AE1
:103E76006480F8EE648098501FAF5CEF3395E0FEE7
:103E8600EF25E0FFEE33FE74222FF58274003EF537
:103E960083E558F0A3E559F0124DB17406255CF59B
:103EA6005C900028E0FEA3E0FFEF4E705CE55EB498
:103EB6000526301423055CAF5CD3EF6480949340F1
:103EC60003755C00C214AF5CEF3395E0FE90003ED4
:103ED600EEF0A3EFF0124DB1E55E64036003023F1E
:103EE6006530147B155CAF5CC3EF6480948050032F
:103EF600755C13C214AF5CEF3395E0FE90003EEEA6
:103F0600F0A3EFF0124DB18056E55EB405263014ED
:103F160023055CAF5CD3EF648094924003755C002C
:103F2600C214AF5CEF3395E0FE90003EEEF0A3EFD7
:103F3600F0124DB1E55EB40326301423155CAF5C78
:103F4600C3EF648094805003755C12C214AF5CEFBB
:103F56003395E0FE90003EEEF0A3EFF0124DB1E592
:103F66005EB40102D214E55E5406FFEF60109000C5
:103F76003EE0FEA3E0FFEF64094E7002C217900117
:103F8600E9E0FEA3E0FF900028E0FCA3E0FDED6F72
:103F96007002EC6E6002C217900028E0FEA3E0FFFC
:103FA6009001E9EEF0A3EFF030A302D21320A30AAA
:0A3FB600301307C213A217B39217CD
:013FC00022DE
:104CAD00124DFA74A0124E127402124E1290001090
:104CBD007C03E0124DD3124E12A3DCF6E0124DD35D
:104CCD00F5F0A3A3E0030354C045F0124E1290007B
:104CDD0014E0124DD3124E12C2B4124DED124DFA14
:104CED0074A0124E1274F0124E12A3E0124E12C2A4
:104CFD00B4124DED22124DFA74A0124E127402121E
:104D0D004E12124DFA74A004124E12900010124E53
:104D1D0037124DDBF0A3124E4A124E37124DDBF017
:104D2D00A3124E4A124E37124DDBF0A3124E4A1209
:104D3D004E37FB543F124DDBF0A3124E4A124E3745
:104D4D00FA541F124DDBF0EB23235403FD124E4496
:104D5D00C2B4124DED124DFA74A0124E1274F0122F
:104D6D004E12124DFA74A004124E12124E37FB540D
:104D7D0003C39D2405838007030201000302012B59
:104D8D00A3F0F5F0124E44C2B4124DED124DFA746B
:104D9D00A0124E1274F0124E12E5F0124E12C2B461
:104DAD00124DED227AA07B807C1E900022124E8A3D
:104DBD00227AA07B80124E52ED900022F07AA0A3B1
:104DCD007C1D124EBF2275F00A84C425F022C0E06E
:0D4DDD00C4540F75F00AA4F5F0D0E0540F97
:104DEA0025F02200D2B5000000D2B4000000002253
:104DFA00124DEDC2B4000000C2B500000022D2B5C7
:104E0A00000000C2B50000227E083392B4124E0898
:104E1A00DEF833D2B40000A2B450040000A2B412E7
:104E2A004E08400122C2B40000124DED227E08A2B3
:104E3A00B43300124E08DEF7C322D2B4124E08224F
:104E4A00C2B4124E08D2B422124DFAEA124E12EB32
:104E5A00124E12124DFAEA04124E12124E37FD1277
:104E6A004E44C2B4124DED22124DFAEA124E12EB22
:104E7A00124E12E6124E1208DCF9C2B4124DED229D
:104E8A00124DFAEA124E12EB124E12E0124E12A311
:104E9A00DCF9C2B4124DED22124DFAEA04124E1296
:104EAA008003124E4A124E37F608DCF6124E44C2FE
:104EBA00B4124DED22124DFAEA04124E1280031278
:104ECA004E4A124E37F0A3DCF6124E44C2B4124DCB
:024EDA00ED22C7
:1049E400202020202531642E2530326420253032C9
:1049F40062753A25303262753A253032627520206C
:104A0400202000202020202532642E2531642025FA
:104A1400303262753A25303262753A253032627529
:104A24002020202000253033642E253164202025C9
:104A34003032642E25316420415A2F454C312020D8
:104A44002000253033642E25316420202530326443
:104A54002E25316420415A2F454C32202020002538
:104A64003033642E2531642020253032642E2531E4
:104A7400642052412F4445432020200025303364D4
:104A84002E2531645720253032642E2531644E2082
:104A94004C4F2F4C412020200025303262752020BD
:104AA400202530326275202025303262753A253057
:104AB4003262753A2530326275202020200025307C
:104AC400352E31662020253032642E253164202095
:104AD400202020202025303264202000202B253067
:104AE40031642E2530316420202B253031642E256D
:104AF40030316420434F522020535450200025303D
:104B040033642E2531642020253032642E2531640F
:104B140020414E5420202531642E2531642000206C
:104B24002020204F20452035204A2046204C20209C
:104B3400202020002020202020202020454D45201A
:104B440020202020202020200020416E74656E6EDD
:104B54006120436F6E74726F6C6C6572200020204C
:104B640020202020207620332E31202020202020B9
:104B74002020002020204A414E4645424D415241CA
:104B840050524D41594A554E4A554C41554753454B
:104B9400504F43544E4F56444543004D4F4F4E20C3
:104BA4002053554E20202043415353494F435947E6
:104BB4004E55535341474954545441555255534CFF
:104BC400454F20202041515541522E52412F4445FA
:104BD40043415A2F454C32415A2F454C3100326DD6
:104BE4003A37303A32333A31333A36636D313047FB
:104BF40000205353492031306269742837323029F8
:104C040020202020202053534931316269742831F7
:104C1400383030292020202020205353493132625B
:104C24006974283336303029202020202020535323
:104C3400495F677261792834303936292020202071
:104C4400202041322D532D532031322062697420AB
:104C540020202020204D414232355F31306269747A
:104C64003130323420202020204D414232355F3112
:104C7400316269743230343820202020204D414282
:104C840032355F3132626974343039362020202065
:104C940020000F0C09010306171D664C03090309C4
:094CA40003090309560101020491
:10002E00E55E640160031257C6200D0302060CC282
:10003E000D30120C900028E0FEA3E0FFEF4E601191
:10004E0090003EE0FEA3E0FFEF64134E600302015A
:10005E00E390003CE0FEA3E0FFC3EF9404EE648067
:10006E00948040030200FCAF1CAE1B12000EEF2466
:10007E0005FFEE3400FE7C007D0A121E128E678F85
:10008E00687B017A00796CC003C002C0017BFF7AE5
:10009E004979E49000DBEBF0A3EAF0A3E9F0AE6758
:1000AE00AF687C007D64121E129000DEEEF0A3EFAE
:1000BE00F0AE67AF687C007D64121E129000E0EC1B
:1000CE00F0A3EDF0900012E0FF9000E2EFF0900050
:1000DE0011E0FF9000E3EFF0900010E0FF9000E4DD
:1000EE00EFF0D001D002D003123758020180AF1CBE
:1000FE00AE1B12000EEF2432FFEE3400FE7C007DAC
:10010E0064121E128E678F687B017A00796CC003B1
:10011E00C002C0017BFF7A4A79079000DBEBF0A3A7
:10012E00EAF0A3E9F0AE67AF687C007D0A121E12FA
:10013E009000DEEEF0A3EFF0AE67AF687C007D0AB4
:10014E00121E129000E0ECF0A3EDF0900012E0FF12
:10015E009000E2EFF0900011E0FF9000E3EFF090DE
:10016E000010E0FF9000E4EFF0D001D002D00312B7
:10017E003758751500D3E515648094825042AF153B
:10018E0090003DE0FE75F003EEA4F58285F083E568
:10019E00822FF582E43583F583E58224E2F582E54C
:1001AE0083344BF583E493FFAE15EEFD3395E0FCFF
:1001BE00746C2DF58274003CF583EFF0051580B557
:1001CE00C3E51B64809480400302059C90006F740D
:1001DE002DF002059C90003EE0FEA3E0FFEF640AC6
:1001EE004E601190003EE0FEA3E0FFEF640B4E6008
:1001FE00030202877B017A00796CC003C002C00142
:10020E007BFF7A4A79299000DBEBF0A3EAF0A3E9B1
:10021E00F090002AE0FEA3E0FF7C007D0A121E1281
:10022E009000DEEEF0A3EFF090002AE0FEA3E0FFD8
:10023E007C007D0A121E129000E0ECF0A3EDF0900F
:10024E00002CE0FEA3E0FF7C007D0A121E1290003F
:10025E00E2EEF0A3EFF090002CE0FEA3E0FF7C00B6
:10026E007D0A121E129000E4ECF0A3EDF0D001D046
:10027E0002D00312375802059C90003EE0FEA3E028
:10028E00FFEF640C4E601190003EE0FEA3E0FFEF26
:10029E00640D4E600302032B7B017A00796CC00360
:1002AE00C002C0017BFF7A4A79469000DBEBF0A3D7
:1002BE00EAF0A3E9F090002EE0FEA3E0FF7C007DC3
:1002CE000A121E129000DEEEF0A3EFF090002EE068
:1002DE00FEA3E0FF7C007D0A121E129000E0ECF0FF
:1002EE00A3EDF0900030E0FEA3E0FF7C007D0A124B
:1002FE001E129000E2EEF0A3EFF0900030E0FEA3AD
:10030E00E0FF7C007D0A121E129000E4ECF0A3EDDB
:10031E00F0D001D002D00312375802059C90003E57
:10032E00E0FEA3E0FFEF640E4E601190003EE0FE93
:10033E00A3E0FFEF640F4E60030203F9900034E078
:10034E00FEA3E0FFEF247CF564EE34FCF563AF64AE
:10035E00AE6312000E7C007D0A121E12C006C0078C
:10036E00AF64AE6312000E7C007D0A121E12900066
:10037E00E4ECF0A3EDF0D007D0069000E2EEF0A38F
:10038E00EFF07B017A00796CC003C002C0017BFFE5
:10039E007A4A79639000DBEBF0A3EAF0A3E9F090E0
:1003AE000032E0FEA3E0FF7C007D0A121E129000D8
:1003BE00DEEEF0A3EFF0900032E0FEA3E0FF7C0053
:1003CE007D0A121E129000E0ECF0A3EDF0D001D0E9
:1003DE0002D003123758C3E5636480948040030251
:1003EE00059C900072742DF002059C90003EE0FE7C
:1003FE00A3E0FFEF64104E601190003EE0FEA3E01C
:10040E00FFEF64114E60030204F6900036E0FEA387
:10041E00E0FFEF24F8F566EE34F8F565900038E06D
:10042E00FEA3E0FFEF247CF564EE34FCF563AF66CB
:10043E00AE6512000E7C007D0A121E12C006C007A9
:10044E00AF66AE6512000E7C007D0A121E12C0044D
:10045E00C005AF64AE6312000E7C007D0A121E1240
:10046E00C006C007AF64AE6312000E7C007D0A1298
:10047E001E129000E4ECF0A3EDF0D007D006900031
:10048E00E2EEF0A3EFF0D005D0049000E0ECF0A384
:10049E00EDF0D007D0069000DEEEF0A3EFF07B017A
:1004AE007A00796CC003C002C0017BFF7A4A798062
:1004BE009000DBEBF0A3EAF0A3E9F0D001D002D07C
:1004CE0003123758C3E5656480948050069000711E
:1004DE007445F0C3E56364809480400302059C90EC
:1004EE0000777453F002059C7B017A00796CC0038F
:1004FE00C002C0017BFF7A4A799D9000DBEBF0A32E
:10050E00EAF0A3E9F0900013E0FF9000DEEFF09028
:10051E000015E0FF9000DFEFF0900012E0FF90007A
:10052E00E0EFF0900011E0FF9000E1EFF09000108E
:10053E00E0FF9000E2EFF0D001D002D00312375866
:10054E00751500D3E515648094825042AF15900066
:10055E0014E0FE75F003EEA4F58285F083E5822F9C
:10056E00F582E43583F583E5822477F582E58334DD
:10057E004BF583E493FFAE15EEFD3395E0FC746E00
:10058E002DF58274003CF583EFF0051580B59000D3
:10059E0028E0FEA3E0FFC3EF9402EE648094805047
:1005AE003290003EE0FEA3E0FFC3EF940AEE6480BB
:1005BE009480401390003EE0FEA3E0FFD3EF941131
:1005CE00EE64809480400C90007E7444F090007F26
:1005DE007445F07F001257D8751500D3E515648069
:1005EE009493501AAF15EF3395E0FE746C2FF5828D
:1005FE0074003EF583E0FF12579F051580DD200E37
:10060E000302080CC20E90003EE0FEA3E0FFC3EF13
:10061E00940AEE64809480401590003EE0FEA3E0C4
:10062E00FFD3EF9411EE648094805002C2129001B9
:10063E00CAE0F8A3E0F9A3E0FAA3E0FB900004E01F
:10064E00FCA3E0FDA3E0FEA3E0FF1219AD12699931
:10065E007B007A00792078411218A47B007A007909
:10066E0000783F1217B3121B068E638F649001CA77
:10067E00E0F8A3E0F9A3E0FAA3E0FB900068E0FC49
:10068E00A3E0FDA3E0FEA3E0FF1219AD1269997B72
:10069E00007A007900783F1217B3121B068E698F0D
:1006AE006A7B017A007984C003C002C0017BFF7AA5
:1006BE004A79C29000DBEBF0A3EAF0A3E9F09001D7
:1006CE00CAE0F8A3E0F9A3E0FAA3E0FB90000CE087
:1006DE00FCA3E0FDA3E0FEA3E0FF1219AD9000DE47
:1006EE00121F5EAE63AF647C007D0A121E12900074
:1006FE00E2EEF0A3EFF0AE63AF647C007D0A121E53
:10070E00129000E4ECF0A3EDF09000E6E569F0A3A2
:10071E00E56AF0D001D002D0031237587F007E0078
:10072E007D007C00900004E0F8A3E0F9A3E0FAA3BA
:10073E00E0FB121A4A500690008A742DF0751500CF
:10074E00D3E515648094855042AF15900029E0FEE4
:10075E0075F006EEA4F58285F083E5822FF582E42E
:10076E003583F583E582249FF582E583344BF5834B
:10077E00E493FFAE15EEFD3395E0FC74902DF582FB
:10078E0074003CF583EFF0051580B5900028E0FE6F
:10079E00A3E0FFC3EF9402EE64809480400E9000BD
:1007AE00967420F09000977420F080217F007E00D8
:1007BE007D007C00900068E0F8A3E0F9A3E0FAA3C6
:1007CE00E0FB121A4A5006900095742DF0E55E6417
:1007DE0001602B7F401257D8751500D3E515648044
:1007EE009493501AAF15EF3395E0FE74842FF58273
:1007FE0074003EF583E0FF12579F051580DD200F34
:10080E0003020917C20F900022E0FEA3E0FFEF24BF
:10081E009CFFEE34FFFE12000E8E658F6690002454
:10082E00E0FEA3E0FFEF249CFFEE34FFFE12000E6D
:10083E008E638F647B017A00799CC003C002C00175
:10084E007BFF7A4A79E09000DBEBF0A3EAF0A3E9B4
:10085E00F0AE65AF667C007D0A121E129000DEEED1
:10086E00F0A3EFF0AE65AF667C007D0A121E12900B
:10087E0000E0ECF0A3EDF0AE63AF647C007D0A12F5
:10088E001E129000E2EEF0A3EFF0AE63AF647C00B8
:10089E007D0A121E129000E4ECF0A3EDF0D001D010
:1008AE0002D003123758900022E0FEA3E0FFC3EF00
:1008BE009464EE64809480500690009D742DF090A8
:1008CE000024E0FEA3E0FFC3EF9464EE6480948006
:1008DE0050069000A3742DF0E55E6401602B7F142A
:1008EE001257D8751500D3E51564809493501AAF3E
:1008FE0015EF3395E0FE749C2FF58274003EF58360
:10090E00E0FF12579F051580DD201003020B19C260
:10091E0010900027E0FFEF904CAA93FFEF3395E085
:10092E00FEAC4EAD4F121E008E438F44AF41AE4013
:10093E0012000E7C007D0A121E12C006C007AF41C7
:10094E00AE4012000E7C007D0A121E129000E4ECE6
:10095E00F0A3EDF0D007D0069000E2EEF0A3EFF09A
:10096E007B017A0079B4C003C002C0017BFF7A4BD1
:10097E0079029000DBEBF0A3EAF0A3E9F0AE45AF0D
:10098E00467C007D0A121E129000DEEEF0A3EFF000
:10099E00AE45AF467C007D0A121E129000E0ECF0D0
:1009AE00A3EDF0AE43AF447C007D0A121E12900000
:1009BE00E6EEF0A3EFF0AE43AF447C007D0A121ECC
:1009CE00129000E8ECF0A3EDF0D001D002D00312AB
:1009DE003758C3E5406480948050069000BA742D59
:1009EE00F0A218B39218E508540CFFEFB4080820D3
:1009FE0018059000C4E4F0E508540CFFEFB40409A8
:100A0E002018069000C47401F0E508540CFFEFB4F2
:100A1E000C093017069000C4742AF0E5085403FF41
:100A2E00EFB402093018069000C37402F0E50854C2
:100A3E0003FFEFB401093018069000C37403F0E50C
:100A4E00085403FFEFB403093017069000C3742A4D
:100A5E00F090003EE0FEA3E0FFEF64124E60030252
:100A6E000AEE751500D3E515648094935042AF15C8
:100A7E0090003BE0FE75F014EEA4F58285F083E560
:100A8E00822FF582E43583F583E58224F5F582E540
:100A9E0083344BF583E493FFAE15EEFD3395E0FC06
:100AAE0074B42DF58274003CF583EFF0051580B516
:100ABE00AE43AF447C007D0A121E12EF2430FF902D
:100ACE0000C5EFF09000C6742EF0AE43AF447C002C
:100ADE007D0A121E12AF05EF2430FF9000C7EFF013
:100AEE007F541257D8751500D3E515648094935032
:100AFE001AAF15EF3395E0FE74B42FF58274003EF5
:100B0E00F583E0FF12579F051580DDE55EB40114F5
:100B1E0090003FE0FFEF904C9693FF1257D812577C
:100B2E00BD1257CF301103020C7C7B017A00796C19
:100B3E00C003C002C0017BFF7A4B79239000DBEB30
:100B4E00F0A3EAF0A3E9F0D001D002D00312375897
:100B5E007B017A007984C003C002C0017BFF7A4B0F
:100B6E0079389000DBEBF0A3EAF0A3E9F0D001D0E6
:100B7E0002D0031237587B017A00799CC003C00261
:100B8E00C0017BFF7A4B794D9000DBEBF0A3EAF0CE
:100B9E00A3E9F0D001D002D0031237587B017A00BE
:100BAE0079B4C003C002C0017BFF7A4B796290001A
:100BBE00DBEBF0A3EAF0A3E9F0D001D002D00312F0
:100BCE0037587F001257D8751500D3E515648094F9
:100BDE0093501AAF15EF3395E0FE746C2FF58274B7
:100BEE00003EF583E0FF12579F051580DD7F401212
:100BFE0057D8751500D3E51564809493501AAF1528
:100C0E00EF3395E0FE74842FF58274003EF583E099
:100C1E00FF12579F051580DD7F141257D8751500EA
:100C2E00D3E51564809493501AAF15EF3395E0FE1B
:100C3E00749C2FF58274003EF583E0FF12579F05DA
:100C4E001580DD7F541257D8751500D3E5156480D5
:100C5E009493501AAF15EF3395E0FE74B42FF582CE
:0F0C6E0074003EF583E0FF12579F051580DD22CD
:1068A100014900014700014800014200C117C1161A
:0268B100C1150F
:10696600752400D3E524648094A75004052480F39D
:0169760022FE
:10697700752500D3E525648094935004052580F39D
:0169870022ED
:10698800752600D3E5266480949E5004052680F37E
:0169980022DC
:105C5100C290126966752C1F752B00E52BD3940732
:105C61005011E52CC313F52CA2D792901269660549
:105C71002B80E8D290126966D2927527037528E8C5
:105C8100752C00309110E52815287002152714FF96
:105C9100AE27EF4E70ED126977752B00E52BD3948B
:105CA100075013126966E52CC313F52C3091034399
:105CB1002C80052B80E6126966AF2C7E00EF752AD9
:105CC10000F5297527037528E8752C00309110E53A
:105CD1002815287002152714FFAE27EF4E70ED121C
:105CE1006977752B00E52BD394075013126966E58C
:105CF1002CC313F52C309103432C80052B80E61225
:105D01006966AF2C7E00EF252AF52AEE3529F529A3
:105D1100C3E529648094805006752900752A00D353
:105D2100E52A940FE5296480948E400675290E7545
:105D31002A0FC29220B20DC3740F952AF52A740E50
:085D41009529F529AE29AF2ACE
:015D49002237
:105E3A00C29412696675321F753100E531D3940731
:105E4A005011E532C313F532A2D79294126966054E
:105E5A003180E8D294126966D296752D03752EE8C0
:105E6A00753200309510E52E152E7002152D14FF8F
:105E7A00AE2DEF4E70ED126977753100E531D3948E
:105E8A00075013126966E532C313F532309503439E
:105E9A003280053180E6126966AF327E00EF7530D6
:105EAA0000F52F752D03752EE8753200309510E533
:105EBA002E152E7002152D14FFAE2DEF4E70ED1219
:105ECA006977753100E531D394075013126966E595
:105EDA0032C313F532309503433280053180E6121E
:105EEA006966AF327E00EF2530F530EE352FF52F9B
:105EFA00C3E52F648094805006752F00753000D357
:105F0A00E530940FE52F6480948E4006752F0E7548
:085F1A00300FC296AE2FAF302C
:015F2200225C
:1068FF00125C518E458F46125E3AC374089FFF7427
:10690F00079EFE12000EC374849FF54174039EF51B
:08691F0040754E00754F012286
:105FE000D290D294D291D2957554007555007550C7
:105FF00000755100753300D3E533648094895049AE
:10600000126988C290C294126988C3E5336480948F
:10601000895004D290D294E5552555F555E554356F
:1060200054F554E5512551F551E5503550F55020C2
:1060300091080555E555700205542095080551E570
:106040005170020550053380AEC290C294754E0067
:10605000754F05AE54AF557C007D05121E008E4570
:106060008F4620B20DC3740B9546F546740E9545C8
:10607000F545C374689551FF74019550FE12000EEA
:10608000C374B49FF551E49EF550AE50AF517C00FF
:096090007D05121E008E408F41B7
:0160990022E4
:10609A00D290D294D291D29575540075550075500C
:1060AA0000755100753400D3E5346480948A5049F0
:1060BA00126988C290C294126988C3E534648094D4
:1060CA008A5004D290D294E5552555F555E55435B4
:1060DA0054F554E5512551F551E5503550F5502008
:1060EA0091080555E555700205542095080551E5B6
:1060FA005170020550053480AEC290C294754E00AC
:10610A00754F02E55525E0F546E55433F54520B2CD
:10611A000DC3740E9546F546740E9545F545C37440
:10612A00849551FF74039550FE12000EC374C29FEA
:10613A00F55174019EF550E55125E0F541E55033DE
:02614A00F5401E
:01614C002230
:1064AF00D290D294D291D2957554007555007550F3
:1064BF0000755100753500D3E5356480948B5049D4
:1064CF00126988C290C294126988C3E535648094BA
:1064DF008B5004D290D294E5552555F555E554359A
:1064EF0054F554E5512551F551E5503550F55020EF
:1064FF0091080555E555700205542095080551E59D
:10650F005170020550053580AEC290C294754E0091
:10651F00754F0185544585554620B20DC3740F95AF
:10652F0046F546740E9545F545C374089551FF74AD
:10653F00079550FE12000EC374849FF54174039E9D
:02654F00F54015
:016551002227
:10581D00D292D296D291D29575540075550075508D
:10582D00007551001269889001EDE4F09001EDE0F2
:10583D00FFD3EF6480948F5044D290D29412698834
:10584D00C290C294126988E5552555F555E5543534
:10585D0054F554E5512551F551E5503550F550208D
:10586D0091080555E555700205542095080551E53B
:10587D0051700205509001EDE004F080AFC290C26E
:10588D0094C292C296754E00754F05E555AE54788B
:10589D0006CEC313CE13D8F9F5558E54E551AE503F
:1058AD007806CEC313CE13D8F9F5518E50AC54AD46
:1058BD0055E4121ACD7B007A00793478441218A47D
:1058CD007B007A00798078441219AD121B067C009A
:1058DD007D05121E008E458F4620B20DC3740B95AB
:1058ED0046F546740E9545F545C3E49551FF740292
:1058FD009550FE12000EC3E49FFD74019EFCEC1248
:10590D001ACD7B007A00793478441218A47B007A82
:10591D0000798078441219AD121B067C007D0512AA
:06592D001E008E408F41B8
:015933002251
:10593400D292D296D291D295755400755500755075
:10594400007551001269889001EEE4F09001EEE0D8
:10595400FFD3EF6480948F5044D290D2941269881C
:10596400C290C294126988E5552555F555E554351C
:1059740054F554E5512551F551E5503550F5502075
:1059840091080555E555700205542095080551E523
:1059940051700205509001EEE004F080AFC290C255
:1059A40094C292C296754E00754F02E555AE547876
:1059B40005CEC313CE13D8F9F5558E54E551AE5028
:1059C4007805CEC313CE13D8F9F5518E50AC54AD2F
:1059D40055E4121ACD7B007A0079E178441218A4B8
:1059E4007B007A00790078451219AD121B06EF2569
:1059F400E0F546EE33F54520B20DC3740E9546F539
:105A040046740E9545F545C3E49551FF74049550CD
:105A1400FE12000EC3E49FFD74029EFCEC121ACD2C
:105A24007B007A0079E178441218A47B007A00792B
:105A34000078451219AD121B06EF25E0F541EE334F
:025A4400F5402B
:015A4600223D
:105A4700D292D296D291D295755400755500755061
:105A5700007551001269889001EFE4F09001EFE0C2
:105A6700FFD3EF6480948F5044D290D29412698808
:105A7700C290C294126988E5552555F555E5543508
:105A870054F554E5512551F551E5503550F5502061
:105A970091080555E555700205542095080551E50F
:105AA70051700205509001EFE004F080AFC290C240
:105AB70094C292C296754E00754F01E554C4F854CE
:105AC700F0C868F554E555C4540F48F555E550C47A
:105AD700F854F0C868F550E551C4540F48F551AC77
:105AE70054AD55E4121ACD7B007A007961784512DE
:105AF70018A47B007A00798078451219AD121B062D
:105B07008E458F4620B20DC3740F9546F546740E29
:105B17009545F545C3E49551FF74089550FE12006D
:105B27000EC3E49FFD74049EFCEC121ACD7B007A31
:105B370000796178451218A47B007A00798078454E
:0A5B47001219AD121B068E408F41AB
:015B51002231
:105B5200D290D294D291D295755400755500755059
:105B620000755100753600D3E5366480948B50532E
:105B7200C290C294753700D3E53764809482500492
:105B8200053780F3C3E5366480948B5004D290D2FB
:105B920094E5552555F555E5543554F554E551250B
:105BA20051F551E5503550F5502091080555E55510
:105BB200700205542095080551E551700205500503
:105BC2003680A4C290C294754E00754F01AF55AE97
:105BD2005412694E8E548F55AF51AE5012694E8E8B
:105BE200508F51AC54AD55E4121ACD7B007A007936
:105BF2006178451218A47B007A00798078451219E1
:105C0200AD121B068E458F4620B20DC3740F95460A
:105C1200F546740E9545F545C3E49551FF74089514
:105C220050FE12000EC3E49FFD74049EFCEC121A97
:105C3200CD7B007A00796178451218A47B007A0046
:0E5C4200798078451219AD121B068E408F41F5
:015C50002231
:1043890075080FE55724F8F54BE55634F8F54AE575
:104399004624F8F54DE54534F8F54CC3E54A648003
:1043A9009480500C7410254BF54B740E354AF54A20
:1043B900C3E54C64809480500C7410254DF54D7400
:1043C9000E354CF54C900038E0FEA3E0FFC3EF94A6
:1043D90084EE648094834025900022E0FEA3E0FFF0
:1043E900E5572FFFE5563EFEEF249CFFEE34FFFE16
:1043F900C3EF9546F539EE9545F5388023900022AF
:10440900E0FEA3E0FFE54B2FFFE54A3EFEEF249CCB
:10441900FFEE34FFFEC3EF954DF539EE954CF538B7
:10442900D3E5539400E5526480948040259000249C
:10443900E0FEA3E0FFE5532FFFE5523EFEEF249C8B
:10444900FFEE34FFFEC3EF9541F53BEE9540F53A9B
:10445900801B900024E0FEA3E0FFEF249CFFEE34D4
:10446900FFFEC3EF9541F53BEE9540F53A20170362
:104479000246BBAE43AF447C007D02121E12D3E557
:10448900399FEE6480F8E53864809840289001F0FF
:10449900E0FFEF20E5067549007548000549AF4979
:1044A900EFD394504003754950E549C3940A4054E9
:1044B90053080E804FAE43AF447C007D02121E129A
:1044C900C3E49FFFE49EFEC3E5399FEE6480F8E5EF
:1044D9003864809850289001F0E0FFEF20E40675D9
:1044E90049007548000549AF49EFD3945040037519
:1044F9004950E549C3940A400B53080D8006754994
:1045090000754800AE43AF447C007D02121E12D3F1
:10451900E53B9FEE6480F8E53A6480984028900175
:10452900F0E0FFEF20E7067547007542000547AF49
:1045390047EFD394504003754750E547C3940A4069
:104549006153080B805CAE43AF447C007D02121EB0
:1045590012C3E49FFFE49EFEC3E53B9FEE6480F82F
:10456900E53A6480985035D3E5419400E54064808C
:10457900948040289001F0E0FFEF20E6067547009F
:104589007542000547AF47EFD39450400375475034
:10459900E547C3940A400B53080780067547007521
:1045A9004200AF39AE3812000E8E3C8F3DC37428DD
:1045B900953DFFE4953CFEEF7802C333CE33CED868
:1045C900F9FFAD487C00C3EF9DF53FEE9CF53EC376
:1045D900E53E648094805006753E00753F00E549CC
:1045E900C39450501DAF497E007C007D7F121E0090
:1045F9007C007D50121E12EF2480FFEF64FFF5FA54
:104609008027C3E53D9428E53C648094805017E5F4
:1046190048C394A050100548C3E53E648094804087
:1046290008853FFA800375FA00AF3BAE3A12000ED7
:104639008E3C8F3DC37428953DFFE4953CFEEF7891
:1046490002C333CE33CED8F9FFAD427C00C3EF9D10
:10465900F53FEE9CF53EC3E53E64809480500675B7
:104669003E00753F00E547C39450501DAF477E009B
:104679007C007D7F121E007C007D50121E12EF24EB
:1046890080FFEF64FFF5FE803BC3E53D9428E53CE0
:10469900648094805017E542C394A050100542C32A
:1046A900E53E64809480401C853FFE801775FE00BE
:1046B900801275490075480075470075420075FA02
:1046C9000075FE00E508C454F0FFEF240FFF9001C8
:0A46D900F0EFF09001F0E0FF8FA079
:0146E30022B4
:1068C7004310000043D8000044A200004511000017
:1068D70045B400004622000000C700C70002000AB6
:1068E7000E0F03840E0F0384000100010000000057
:0868F700000000000000000099
:1068B300011400011663011200011700011A00C13F
:0368C3000CC18B7A
:03000300025F2376
:105F2300C0E0C083C08263A201C083C082C0D075B9
:105F3300D000C006C007200B4F200C4CD2B330B3A7
:105F4300020512051AAF1AC3EF64809488401CAF90
:105F530017EF3395E0FE74402FF58274003EF5830E
:105F6300E512F07512000517751A00E5122512F5F2
:105F730012C3E51764809484404F751700D20C90C8
:105F83000048E0FF8F128041200B3E300C3BE512AE
:105F93002512F512A2D792B3051AAF1AC3EF648084
:105FA3009488401A0517AF17EF3395E0FE74482F16
:105FB300F58274003EF583E0FF8F12751A00C3E586
:105FC30017648094A04002D20BD007D006D0D0D063
:0D5FD30082D08363A201D082D083D0E0325F
:104EDC00900048E556F0A3E557F0E5532484FFE530
:104EEC00523403FE90004AEEF0A3EFF090004CE534
:104EFC0045F0A3E546F0E5412484FFE5403403FE8C
:104F0C0090004EEEF0A3EFF0E50B2484FFE50A349D
:104F1C0003FE900050EEF0A3EFF0900022E0FEA311
:104F2C00E0FF900052EEF0A3EFF0900024E0FEA31F
:104F3C00E0FF900054EEF0A3EFF0900028E0FEA309
:104F4C00E0FF900056EEF0A3EFF0900058E543F030
:104F5C00A3E544F030170B90005AE4F0A37401F071
:104F6C00800890005AE4F0A3E4F0900015E0FFEF05
:104F7C003395E0FE90005CEEF0A3EFF0900014E0AF
:104F8C00FFEF3395E0FE90005EEEF0A3EFF09000A3
:104F9C0013E0FFEF3395E0FE900060EEF0A3EFF02E
:104FAC00900012E0FFEF3395E0FE900062EEF0A36C
:104FBC00EFF0900011E0FFEF3395E0FE900064EE0F
:104FCC00F0A3EFF0900041E0F516900040E4F0A360
:104FDC007463F0C3E5166480948840030250C1C327
:104FEC00E5166480948050030250C1900042E0F5B5
:104FFC0018A3E0F519AF16EF3395E0FEEF25E0FFAF
:10500C00EE33FE74DF2FF58274683EF583E493FE75
:10501C00740193FFD3E5199FEE6480F8E518648062
:10502C00984021AF16EF3395E0FEEF25E0FFEE330D
:10503C00FE74DF2FF58274683EF583E493F51874E3
:10504C000193F519AF16EF3395E0FEEF25E0FFEE77
:10505C0033FE74EF2FF58274683EF583E493FE748F
:10506C000193FFC3E5199FEE6480F8E518648098FE
:10507C005021AF16EF3395E0FEEF25E0FFEE33FE47
:10508C0074EF2FF58274683EF583E493F518740180
:10509C0093F519AF16EF3395E0FEEF25E0FFEE33F5
:1050AC00FE74222FF58274003EF583E518F0A3E51B
:1050BC0019F0124DB1E516B40805A217B3921722D8
:03002B0002614D22
:10614D00C0E0C0F0C083C08263A201C083C082C022
:10615D00D075D000C000C001C002C003C004C0058E
:10616D00C006C007C2CF75A61E75A6E11509AF09F9
:10617D00EF705E75090490003AE0FEA3E0FFEF8E2C
:10618D00F0121FE161B5000061BA000161BF0002AC
:10619D0061C4000361C9000461CE000561D300062E
:1061AD0061D80007000061DB125FE0802112609A68
:1061BD00801C1264AF8017125B5280121268FF8030
:1061CD000D12581D80081259348003125A4712437C
:1061DD0089D007D006D005D004D003D002D001D08D
:1061ED0000D0D0D082D08363A201D082D083D0F0F2
:0361FD00D0E032BD
:03002300026797DA
:10679700C0E0C0F0C083C08263A201C083C082C0D2
:1067A700D075D000C000C001C002C003C004C0053E
:1067B700C006C007C2AC30981AC298E599B43F0327
:1067C7001250CCE599B4210B1252B2D20DD20ED28F
:1067D7000FD210C299D2ACD007D006D005D004D0C2
:1067E70003D002D001D000D0D0D082D08363A201E1
:0967F700D082D083D0F0D0E03252
:03000B000262008E
:10620000C0E0C0F0C083C08263A201C083C082C06E
:10621000D075D000C000C001C002C003C004C005DA
:10622000C006C007758A00758C4C75A61E75A6E160
:106230000514AF14C3EF6480948A4016300B1375B5
:106240001400751700751A00C20CC20B75120012EB
:106250004EDCE51375F007121D86AFF0EF701E12CD
:106260003B76301104D20DD210E55E600730110488
:10627000D20ED20F12002E124D02124DBE1513AFC8
:1062800013EF700C75134ED211301104D20ED20FD1
:10629000D007D006D005D004D003D002D001D00062
:1062A000D0D0D082D08363A201D082D083D0F0D06E
:0262B000E032DA
:10217B00758FFF758921758DFF438780759850D2B8
:10218B008CD28ED2CA75CB4C75CA0043B81143B7EB
:10219B0021D28875D90243D84075DA4275DE42C226
:1021AB00117513467509017F021257671257B475E3
:1021BB005F00900040E4F0A37463F020A00312676B
:1021CB001D75A8B275A707E55E70FC900036E0FCA4
:1021DB00A3E0FDEC121ACD7B007A00792078411236
:1021EB0019AD7B007A00793478C31217B39001CA0A
:1021FB00E0F8A3E0F9A3E0FAA3E0FB1218A4900027
:10220B001E121F5E900038E0FCA3E0FDEC121ACD0D
:10221B007B007A00792078411219AD7B007A007926
:10222B00B478C21217B39001CAE0F8A3E0F9A3E0A7
:10223B00FAA3E0FB1218A490001A121F5E90001173
:10224B00E0FCEC121AD27B007A0079B478441219B4
:10225B00ADC004C005C006C007900012E0FCEC1234
:10226B001AD27B007A0079C078411219ADA804A963
:10227B0005AA06AB07D007D006D005D0041217B3BA
:10228B00C004C005C006C007900010E0FCEC121A99
:10229B00D27B007AC079A878471219ADA804A9059A
:1022AB00AA06AB07D007D006D005D0041217B390FF
:1022BB000044121F5E900014E0FFEF3395E0FEFD2B
:1022CB00FCEF2409FFEE3400FEED3400FDEC34008E
:1022DB00FC7B0C7A0079007800126800A804A90531
:1022EB00AA06AB07900015E0FFEF3395E0FEFDFC6F
:1022FB00EF24D0FFEE3407FEED3400FDEC3400FC90
:10230B00EB2FFFEA3EFEE93DFDE83CFC7B077A0044
:10231B0079007800121E5E7B047A00790078001237
:10232B006800C004C005C006C007900015E0FFEFB1
:10233B003395E0FEFDFC7B6F7A0179007800121E6D
:10234B005ED003D002D001D000C3EF9BFFEE9AFE0C
:10235B00ED99FDEC98FCC004C005C006C0079000C9
:10236B0014E0FFEF3395E0FEFDFC7B137A0179005F
:10237B007800121E5E7B097A0079007800126800E3
:10238B00A804A905AA06AB07D007D006D005D00430
:10239B00EB2FFBEA3EFAE93DF9E83CF8900013E03D
:1023AB00FFEF3395E0FEFDFCEB2FFFEA3EFEE93D30
:1023BB00FDE83CFCEF247AF511EE34E0F510ED343A
:1023CB0000F50FEC3400F50E900028E0FEA3E0FFC3
:1023DB00EF64014E70487B017A007908C003C0029C
:1023EB00C0017B017A007968900193EBF0A3EAF0CE
:1023FB00A3E9F0AF11AE10AD0FAC0E900196121F0A
:10240B005E900044E0FCA3E0FDA3E0FEA3E0FF90A0
:10241B00019A121F5ED001D002D003123FC190006F
:10242B0028E0FEA3E0FFEF4E60030226007B017A5B
:10243B00007908C003C002C0017B017A0079689063
:10244B00010BEBF0A3EAF0A3E9F0AF11AE10AD0F67
:10245B00AC0E90010E121F5E900044E0FCA3E0FD59
:10246B00A3E0FEA3E0FF900112121F5ED001D00289
:10247B00D0031229D590001AE0FCA3E0FDA3E0FEE7
:10248B00A3E0FF12549E7B547AE3794578401218EF
:10249B00A4C004C005C006C007900016E0FCA3E072
:1024AB00FDA3E0FEA3E0FF1254B4A804A905AA06FD
:1024BB00AB07D007D006D005D0041218A4C004C0B7
:1024CB0005C006C007900068E0FCA3E0FDA3E0FE9A
:1024DB00A3E0FF12549EA804A905AA06AB07D007D8
:1024EB00D006D005D0041218A4C004C005C006C085
:1024FB0007AF11AE10AD0FAC0EC004C005C006C0C7
:10250B00077FAB7EAA7D2A7C3C900044E0F8A3E0D9
:10251B00F9A3E0FAA3E0FB1217B3900146121F5E7A
:10252B00D007D006D005D004120C7DC004C005C066
:10253B0006C007AF11AE10AD0FAC0EC004C005C086
:10254B0006C0077FAB7EAA7D2A7CBC900044E0F8D6
:10255B00A3E0F9A3E0FAA3E0FB1217B39001461234
:10256B001F5ED007D006D005D004120C7DD003D04F
:10257B0002D001D0001217AF7B007A007987784325
:10258B001219ADA804A905AA06AB07D007D006D02F
:10259B0005D0041217B37B007A00797A78441218AD
:1025AB00A4121B068E0C8F0DAC0CAD0DEC121ACDBC
:1025BB00C004C005C006C00790003CE0FEA3E0FFCE
:1025CB00EF7802C333CE33CED8F9FF74C72FF58221
:1025DB0074683EF583121F2ED007D006D005D004A9
:1025EB001218A47B007A00797A78441219AD121B69
:1025FB00068E1B8F1C900028E0FEA3E0FFEF640209
:10260B004E7014900068121F6A3F82D0E59000084C
:10261B00121F6A40C39DB2900028E0FEA3E0FFEFBB
:10262B0064034E7014900068121F6A3F3566CF909A
:10263B000008121F6A40A73B64900028E0FEA3E04D
:10264B00FFEF64044E7014900068121F6ABF018F75
:10265B00C5900008121F6A40953F7D900028E0FE50
:10266B00A3E0FFEF64054E7014900068121F6A3EE2
:10267B00C44D01900008121F6A3FB91687900028BD
:10268B00E0FEA3E0FFEF64064E7014900068121F8B
:10269B006A3F32B6AE900008121F6A401F2B0290A1
:1026AB000028E0FEA3E0FFEF64074E701490006873
:1026BB00121F6A00000000900008121F6A40BC7ACB
:1026CB00E1900028E0FEA3E0FFEF64084E706790F6
:1026DB000032E0FCA3E0FDEC121ACD7B007A00790E
:1026EB002078411219AD9001CAE0F8A3E0F9A3E0FC
:1026FB00FAA3E0FB1218A4900008121F5E9000349E
:10270B00E0FCA3E0FDEC121ACD7B007A0079207877
:10271B00411219AD7B007A0079B478C21217B390CD
:10272B0001CAE0F8A3E0F9A3E0FAA3E0FB1218A4B6
:10273B00900068121F5E900028E0FEA3E0FFC3EF3D
:10274B009409EE648094804003022854900044E086
:10275B00FCA3E0FDA3E0FEA3E0FFC004C005C006A0
:10276B00C007AF11AE10AD0FAC0E9001B6121F5ECD
:10277B00D007D006D005D0041246E4900170121F8A
:10278B005E7B017A00790CC003C002C0017B017A29
:10279B0000790090016DEBF0A3EAF0A3E9F0900053
:1027AB0008E0FCA3E0FDA3E0FEA3E0FF90017412A0
:1027BB001F5E900068E0FCA3E0FDA3E0FEA3E0FF3A
:1027CB00900178121F5ED001D002D0031231DC9041
:1027DB000028E0FEA3E0FFEF4E705A900000E0FCF3
:1027EB00A3E0FDA3E0FEA3E0FF12549E7B007A5012
:1027FB0079C778451218A4C004C005C006C007905D
:10280B0000D0121F6A48B98C00D007D006D005D073
:10281B00041265EFA804A905AA06AB07900000E017
:10282B00FCA3E0FDA3E0FEA3E0FF1217AF900004B2
:10283B00121F5E8014900000E0FCA3E0FDA3E0FEFD
:10284B00A3E0FF900004121F5E900028E0FEA3E0BF
:10285B00FFEF64094E705C90002EE0FCA3E0FDECF2
:10286B00121ACD7B007A00792078411219AD9001B4
:10287B00CAE0F8A3E0F9A3E0FAA3E0FB1218A490D6
:10288B00000C121F5E900030E0FCA3E0FDEC121A6E
:10289B00CD7B007A00792078411219AD9001CAE006
:1028AB00F8A3E0F9A3E0FAA3E0FB1218A49000044C
:1028BB00121F5E900028E0FEA3E0FFEF640A4E704B
:1028CB005C90002AE0FCA3E0FDEC121ACD7B007AB1
:1028DB0000792078411219AD9001CAE0F8A3E0F914
:1028EB00A3E0FAA3E0FB1218A490000C121F5E9059
:1028FB00002CE0FCA3E0FDEC121ACD7B007A0079F2
:10290B002078411219AD9001CAE0F8A3E0F9A3E0D9
:10291B00FAA3E0FB1218A4900004121F5E9001CAE8
:10292B00E0F8A3E0F9A3E0FAA3E0FB90000CE0FCD5
:10293B00A3E0FDA3E0FEA3E0FF1219AD7BCD7ACCA3
:10294B00794C783D1217B37B007A007920784112CD
:10295B0018A4121B068E568F579001CAE0F8A3E0FD
:10296B00F9A3E0FAA3E0FB900004E0FCA3E0FDA3D5
:10297B00E0FEA3E0FF1219AD7BCD7ACC794C783D0C
:10298B001217B37B007A00792078411218A4121B1E
:10299B00068E528F537F007E007D207C4190006815
:1029AB00E0F8A3E0F9A3E0FAA3E0FB1218A490016E
:1029BB00CAE0F8A3E0F9A3E0FAA3E0FB1219AD1209
:0A29CB001B068E0A8F0B0221D22298
:10570000EFC0E0C283740F125735743012573F74E4
:1057100005125735743012573F74011257357430E3
:1057200012573F7401125735D0E0146002740844D8
:105730002012574D227D000000DDFCD5E0F72254F9
:10574000F053800F4280C282D283C28322C2828001
:1057500002D282C0E012575BD0E0C454F053800FF5
:105760004280D283C28322125700125799740612C4
:10577000574D125799740E12574D125799740112C2
:10578000574D125799744012574D1257E6125799B8
:10579000748012574D1257C622740A12573522EFE1
:1057A000C0E0125799D0E012575122125799740253
:1057B00012574D22125799740112574D22125799C0
:1057C000740E12574D22125799740C12574D221213
:1057D0005799740F12574D22EFC0E0125799D0E03D
:1057E000448012574D229057F57E28E493FF1257BC
:1057F0009FA3DEF7220004040E0E1F1F00001F1FD0
:105800000E0E04040000101C1F1C100000000107F5
:0D5810001F070100000E11171917110E00DF
:10694E007A107B00EE6BFB8BF053F080ABF033EFE5
:08695E0033FFEE33FEDAEE22F6
:10668C009001EBEEF0A3EFF09001EBE0FEA3E0FF46
:10669C007C037DE8121E12EF2430F5993099FDC26F
:1066AC00999001EBE0FEA3E0FF7C037DE8121E1243
:1066BC007E007F64CFCDCFCECCCE121E12EF243015
:1066CC00F5993099FDC2999001EBE0FEA3E0FF7CB7
:1066DC00007D64121E127E007F0ACFCDCFCECCCEB1
:1066EC00121E12EF2430F5993099FDC2999001EBEE
:1066FC00E0FEA3E0FF7C007D0A121E12AF05EF2422
:10670C0030F5993099FDC2997599003099FDC2996F
:01671C00225A
:1050CC009001E1121F6A000186A020983E9001E138
:1050DC00E0FCA3E0FDA3E0FEA3E0FFEC4D4E4F602F
:1050EC002A9001E1E0FCA3E0FDA3E0FEA3E0FF7B3E
:1050FC00FF7AFF79FF78FFEF2BFFEE3AFEED39FDDB
:10510C00EC38FC9001E1121F5E80BFC298AF99EFA2
:10511C00121FBB517161517D625189635191645170
:10512C009D6551A96651B56751C16851CD6951D979
:10513C006A51E56B51F16C51FD6D52096E52176F4E
:10514C00521F70522D71523572524373524B74521E
:10515C005E75526C76527A7752887852967952A450
:10516C007A000052B1900022E0FEA3E0FF12668CA0
:10517C0022900024E0FEA3E0FF12668C22AF44AE26
:10518C004312668C22900028E0FEA3E0FF12668C8E
:10519C002290002AE0FEA3E0FF12668C2290002CE5
:1051AC00E0FEA3E0FF12668C2290002EE0FEA3E04E
:1051BC00FF12668C22900030E0FEA3E0FF12668C9A
:1051CC0022900032E0FEA3E0FF12668C22900034A5
:1051DC00E0FEA3E0FF12668C22900036E0FEA3E016
:1051EC00FF12668C22900038E0FEA3E0FF12668C62
:1051FC002290003AE0FEA3E0FF12668C22E50D241B
:10520C0088FFE50C3413FE12668C22AF46AE4512B5
:10521C00668C22E5412484FFE5403403FE12668C43
:10522C0022AF57AE5612668C22E5532484FFE5520A
:10523C003403FE12668C22AF0BAE0A12668C22303F
:10524C0017087F017E0012668C227F007E0012669A
:10525C008C22900010E0FFEF3395E0FE12668C225A
:10526C00900011E0FFEF3395E0FE12668C22900067
:10527C0012E0FFEF3395E0FE12668C22900013E0F3
:10528C00FFEF3395E0FE12668C22900014E0FFEFE6
:10529C003395E0FE12668C22900015E0FFEF3395FB
:0552AC00E0FE12668C1B
:0152B10022DA
:10640A009001D6E4F0A3E4F09001DCE4F09001DC22
:10641A00E0FFD3EF6480948340030264A69001D81E
:10642A00121F6A000186A020983E9001D8E0FCA3C2
:10643A00E0FDA3E0FEA3E0FFEC4D4E4F602A900181
:10644A00D8E0FCA3E0FDA3E0FEA3E0FF7BFF7AFF18
:10645A0079FF78FFEF2BFFEE3AFEED39FDEC38FCC1
:10646A009001D8121F5E80BFC2989001D6E0FEA3A9
:10647A00E0FF7C007D0A121E00AD997C00EF2DFF23
:10648A00EE3CFEEF24D0FFEE34FFFE9001D6EEF094
:10649A00A3EFF09001DCE004F00264179001D6E06B
:0464AA00FEA3E0FF6E
:0164AE0022CB
:1052B2009001E5121F6A000186A020983E9001E548
:1052C200E0FCA3E0FDA3E0FEA3E0FFEC4D4E4F6047
:1052D2002A9001E5E0FCA3E0FDA3E0FEA3E0FF7B52
:1052E200FF7AFF79FF78FFEF2BFFEE3AFEED39FDF3
:1052F200EC38FC9001E5121F5E80BFC298AF99EFB7
:10530200121FBB5345615354625363635372645318
:105312008165539066539F6753AE6853BD6953CC02
:105322006A53DB6B53EA6C53F96D540874540E756F
:10533200541A76542677543278543E79544A7A0075
:1053420000545512640A900022EEF0A3EFF0124DC1
:10535200B12212640A900024EEF0A3EFF0124DB1D4
:105362002212640A900026EEF0A3EFF0124DB12251
:1053720012640A900028EEF0A3EFF0124DB122124F
:10538200640A90002AEEF0A3EFF0124DB1221264EB
:105392000A90002CEEF0A3EFF0124DB12212640A33
:1053A20090002EEEF0A3EFF0124DB12212640A909B
:1053B2000030EEF0A3EFF0124DB12212640A900019
:1053C20032EEF0A3EFF0124DB12212640A900034D3
:1053D200EEF0A3EFF0124DB12212640A900036EE05
:1053E200F0A3EFF0124DB12212640A900038EEF0F1
:1053F200A3EFF0124DB12212640A90003AEEF0A32C
:10540200EFF0124DB122A217B392172212640A9042
:105412000010EFF0124CAD2212640A900011EFF06E
:10542200124CAD2212640A900012EFF0124CAD221F
:1054320012640A900013EFF0124CAD2212640A902B
:105442000014EFF0124CAD2212640A900015EFF036
:03545200124CAD4C
:015455002234
:1017AC00021B72E86480F8E933E83360110460F0DE
:1017BC00ED33EC337009E8FCE9FDEAFEEBFF2204A3
:1017CC0060DED3EB9FEA9EE99DE8C2E78CF0C2F79E
:1017DC0095F0400CE8CCF8E9CDF9EACEFAEBCFFB6A
:1017EC00121B3D85D0F05804700320D5B3E804706B
:1017FC00075002B2D5021B7C92D5EC0460F7E4CC06
:10180C00C0E0C398F8603B94186008400DD0E0FB32
:10181C00021B54E4FBFAC9FC8028E830E406E4C956
:10182C00FBE4CAFCE830E305E4C9CACBFCE8540786
:10183C006010F8C3E913F9EA13FAEB13FBEC13FC91
:10184C00D8F130F52FC3E49CFCEF9BFFEE9AFEED34
:10185C0099FDD0E0FBEF4E4D4C701222DB03021BC6
:10186C0079EC2CFCEF33FFEE33FEED33FDED30E77E
:10187C00EB021B54EF2BFFEE3AFEED39FDD0E0FBF3
:10188C0050130BBB0003021B7CED13FDEE13FEEF9C
:08189C0013FFEC13FC021B54C6
:1018A400EC4D6011E8497017ED33EC3304600DE43E
:1018B400FCFFFEFD22E933E8330470F8021B7212C8
:1018C4001B3D58046009E4CC2481500628500902C9
:1018D4001B7C284003021B79C0E0EB4A7044B980AA
:1018E40006D0E0FB021B68EF4E701CBD8008EBFFC6
:1018F400EAFEE9FD80EBE98DF0A4FEE5F002198D26
:10190400E9CDF9EAFEEBFFEF89F0A4FCE5F0CE891E
:10191400F0A42EFFE435F0CD89F0A42DFEE435F0DB
:101924008067EF4E7005BD80D780C3EF8BF0A4AC09
:10193400F0EE8BF0A42CFCE435F0F8EF8AF0A42C44
:10194400E5F038FCE433CB8DF0A42CFCE5F03BF857
:10195400EE8AF0A42CFCE5F038F8E433CF89F0A447
:101964002CFCE5F038CF3400CE89F0A42FFFE5F04D
:101974003EFEE433C98DF0A42EFEE5F039CD8AF0A5
:10198400A42FFFE5F03EFEE43DFD33D0E0FB50071D
:101994000BBB000F021B7CEC2CFCEF33FFEE33FE81
:0619A400ED33FD021B54AF
:1019AA00021B7CEC5D046005E859047003021B729B
:1019BA00121B3D580460F6EC4860F2EC7004FDFE20
:1019CA00FF22C860DB2481C85009C3986002500610
:1019DA00021B799850CAF582E9294B4A7005AB82F5
:1019EA00021B6875F0007C1A7880C3EF9BEE9AEDB3
:1019FA0099400DC3EF9BFFEE9AFEED99FDE842F088
:101A0A00DC23ACF0D0E0FFD0E0FED0E0FDAB8220DA
:101A1A00E7101BEB60BAEC2CFCEF33FFEE33FEED64
:101A2A0033FD021B54E803F830E705C0F075F000F7
:101A3A00EF2FFFEE33FEED33FD40B830E7C280AA48
:101A4A0074F8CC6480CCC86480C8F582046043C34F
:101A5A00EB9FF5F0EA9E42F0E99D42F0E89C45F0E2
:101A6A0060305018E5825FFFE582F42B5582FB5007
:101A7A00210ABA001D09B90019088016E5825BFB24
:101A8A00E582F42F5582FF50090EBE00050DBD00F8
:101A9A00010CC3EB9FF5F0EA9E42F0E99D42F0E8A3
:0D1AAA009C45F06007CC4820E701B3EC221A
:101AB700ED33EC33600A047003BD8004ECB2E7FC3D
:011AC70022FC
:101AC80075F020800E75F010800575F0087D007E99
:101AD800007F003392D530D503121EADEC33401091
:101AE800EF33FFEE33FEED33FDEC33FCD5F0ED22A2
:0E1AF800E5F0247EA2D513CC92E7CDCEFF22DE
:101B0600EDD2E7CD33EC3392D524814006E4FFFED7
:101B1600FDFC22FCE4CFCECDCC24E0501174FF8036
:101B2600EDC3CC13CCCD13CDCE13CECF13CF0470D3
:071B3600F030D5DE021EAD08
:1036F300E56B24DBF582E43400F583E0056B22906F
:1037030000D83009039000DBE475F001121F9B021F
:103713001DA82002E97F2ED2028018EF540F2490B7
:10372300D43440D4FF30060BEF24BFB41A00500347
:103733002461FFE56C6002156C056FE56F7002058F
:103743006E30090E9000D8E475F001121F9BEF0252
:103753001DEE0269277403D2098003E4C209F56BE5
:103763009000D8121FB2E4F56CF56EF56FE56C604E
:10377300077F2012373680F5756DFFC203C202C280
:1037830004C205C207C208C20A123702FF700D3015
:1037930009057F00123747AF6FAE6E22B4255FC2B3
:1037A300D5C206123702FF24D0B40A00501A75F0AE
:1037B3000A786C30D50508B6FF0106C6A426F620A4
:1037C300D5047002D20580D924CFB41A00EF500477
:1037D300C2E5D206023A39D20380C6D20280C0D2F1
:1037E3000480BCD2D580BAD20780B47F201237368A
:1037F3002004077401B56C0040F11236F3FF123751
:1038030036023770D20AD20880951236F3FB12368D
:10381300F3FA1236F3F94A4B700679377A3B7BFF9A
:1038230020042EE56C602A7E008E82758300121DB3
:10383300C160060EEE656D70F0C2D5EBC0E0EAC064
:10384300E0E9C0E0EE123A9AD0E0F9D0E0FAD0E035
:10385300FB121DA8FF60AAEBC0E0EAC0E0E9C0E0EC
:10386300123736D0E02401F9D0E03400FAD0E0FB7F
:10387300E56D0460DCD56DD98087D20480A2123A4D
:103883007C60F7E56D700104121B87A96D600DE57F
:103893006D600914F56D123B24EF60F3EA30E70223
:1038A300F404C3995079EAF4256D0430E701E40484
:1038B300F56D800D123A7C60C1EA056D256D121B12
:1038C30087EA900107F030E701E4256D04D56D0424
:1038D30020070114123A9AE4C0E0123B2490010736
:1038E300E0601320E70714F012371E802204F0D0A3
:1038F300E014C0E07F0012371EE56D600712371534
:10390300156D800B300703123715D0E0023770D0E6
:10391300E00480C4123A7C609EE56D04121B87901C
:103923000107EAF0E56D2007026001042404123A5E
:013933009AF9
:1039340074FF04C0E0123B2412371EE56D20070219
:103944006003123715D0E0B56DE87F451237289033
:103954000107E07F2B30E7047F2DF404C0E0123729
:1039640036D0E075F00A84C0F012371FD0E0123769
:103974001F023770791080027908C208C20A8008D1
:10398400D2D5790A8004790AC2D5E56D047002F5AE
:103994006DE4FAFDFEFF1236F3FC7B0820031312DC
:1039A40036F3FD7B1030020A1236F3FE1236F3FFB3
:1039B4007B20EC3382D592D55013C3E43002069FAA
:1039C400FFE49EFEE42003039DFDE49CFCE4CBF8AD
:1039D400C203EC700CCFCECDCCE824F8F870F380A1
:1039E40017C3EF33FFEE33FEED33FDEC33FCEB3363
:1039F400FB994002FB0FD8E9EB300305F8D0E0C493
:103A040048B203C0E00AEC4D4E4F78207B0070C2F0
:103A1400EAB56D0040BCC0E0123A9CD0F0D0E02082
:103A24000304C4C0E0C4B203C0F012371FD0F0D501
:103A3400F0EB023770121FBB380D5339785837DE5C
:103A44004C37DA42397C4F39844439844937F3435B
:103A5400398A5538B7463917453881473B57503767
:103A6400E22D37E62E38092B37EA233807203B406E
:103A74002A37A24800003801E56DB4FF03756D06CE
:103A84001236F3FC1236F3FD1236F3FE1236F3FF50
:103A9400900100021BC4790AA2D52005143007093D
:103AA400B910020404B9080104A2D5200802500187
:103AB400042004689204B56C005034C0E07F2030C8
:103AC40005197F30A20472087207500F123AF3C22C
:103AD40004C208C207C20A7F30800F300703E9C05E
:103AE400E0123736300703D0E0F9D0E0B56CCC30C3
:103AF40007177F30B9100C1237367F583006077F0E
:103B0400788003B908031237363004057F2D023755
:103B1400367F20200AF87F2B2008F322920480CFDE
:103B24007F00B40700500B2400F582E43401F583D0
:103B3400E0FF22286E756C6C2900D2031236F33034
:103B440003F8C203786C30D50108F60237A22D5071
:103B54004349581236F32403B405004001E4903B72
:103B64005293123727743A123727D205756C040220
:023B740039789E
:0D699900ED33EC3360065004EC6480FC220A
:10635E00021B7222EDA2E7D2E7F9EC3340F260F3B2
:10636E00B4FF08ED547F70E8021B7CF82481C2E074
:10637E00C0E0F40428FAC313FCED92E7FD9000CCC4
:10638E00121F5EEEA2E7E9BA7F02C3133400940037
:10639E00FA75F091A4E5F013F494FE8AF0A433E5B7
:1063AE00F033248CD313FDE492E7FE7F007C3F751F
:1063BE008302ECC0E0F8EDC0E0F9EEC0E0FAEFC009
:1063CE00E0FB8583F09000CC121F0685F083121936
:1063DE00ADD0E0FBD0E0FAD0E0F9D0E0F81217B380
:1063EE00ED6480FD30E7011CD583C7ED33CC33F867
:0C63FE00D0E0A2E71328C313CC13FD224B
:1065EF009000CC121F5E9000D0E0F8A3E0F9A3E07A
:1065FF00FAA3E0FB9000CCE0FCA3E0FDA3E0FEA338
:10660F00E0FF1219AD1255FE9000CC121F5E9000E4
:10661F00D0E030E7599000CCE0FCA3E0FDA3E0FE12
:10662F00A3E0FFECC0E0EDC0E0EEC0E0EFC0E0E4BF
:10663F00FFFEFDFC9000CCE0F8A3E0F9A3E0FAA385
:10664F00E0FB121A4A7BDB600250087A0F79497817
:10665F004080067A0F794978C0D0E0FFD0E0FED0B5
:10666F00E0FDD0E0FC1217B39000CC121F5E90003B
:0D667F00CCE0FCA3E0FDA3E0FEA3E0FF22C1
:105456003A70FA83BCAAE9E43E81E0F8BF9DE9E62A
:105466003F80000039283C1ABB9969663DA335E3A5
:10547600BF255DE73FC90FDB418DDBCCC44936EE66
:1054860045C9913FC5B0F83D3F800000C317F534CC
:10549600452FFA73C60AFDDD12555F04A2E192009C
:1054A6001420E0159054567404121CC9803012550D
:1054B6005F30E102B20020E0EBA883A9829000CC25
:1054C600121F5E8982888390546A7404121CC985EF
:1054D60082F09000CC121F2285F0821218A4ED4CA7
:1054E6006007300004EC6480FC2212555FC0E0A81F
:1054F60083A9829000CC121F5E8982888390548E85
:105506007403121CC98582F09000CC121F2285F00C
:10551600821218A49000CCE0CCF0A3E0CDF0A3E07A
:10552600CEF0A3E0CFF090547E7403121CC9D08253
:105536008582F09000CC121F2285F082E58230E051
:10554600071219ADB2008096EFCBFFEECAFEEDC989
:10555600FDECC8FC1219AD8085ED33EC547FCC33DD
:10556600920024605007D0E0D0E0021B727B837A61
:10557600F97922783E1218A4EDF933ECF833248138
:105586005011EFFBEEFA121B06121AC8ECB2E7FC3A
:105596001217B3ED33EC33602F2403F8C313FCED7D
:1055A60092E7FDE82481E4501FECF8EDF9EEFAEFFE
:1055B600FB121B06EF04C2E0FCF582121AD2ECB213
:1055C600E7FC1217B3E58203FAED33EC33600714F8
:0855D60013FCED92E7FDEA224F
:1055DE00BE1249253E4CCCCDBEAAAAAB3F800000E0
:1055EE003E7ADBB03EED63383F24BC7D3F490FDB96
:1055FE00ED33ECC2E7CC339200B4FF13ED547F6071
:10560E0003021B727FDB7E0F7DC97C3F0256F3C205
:10561E0001C3947F401E7007EDD2E794904015EFC2
:10562E00FBEEFAEDF9ECF87F007E007D807C3F12F8
:10563E0019ADD201ED33EC33248430E705E4C0E03C
:10564E00806B04FAEDD2E754F0C333DAFD5407341D
:10565E00002323C0E0CCC0E0F8EDC0E0F9EEC0E0DE
:10566E00FAEFC0E0FBE4121AD2EC24FEFC9000D458
:10567E00121F5E1218A47B007A007980783F1217F1
:10568E00B39000D4E0B2E7CCF0A3E0CDF0A3E0CE2F
:10569E00F0A3E0CFF0D0E0FBD0E0FAD0E0F9D0E01C
:1056AE00F81217B39000D4121F221219AD9000D425
:1056BE00121F5E9055DE7403121CC99000D4121F87
:1056CE00221218A4D0E0600F24EAF582E43455F5D6
:1056DE0083121F2E1217B330010B7BDB7A0F79C9A1
:1056EE0078BF1217B3ED33EC336006ECA20092E7ED
:0256FE00FC228C
:105D4A009000CC121F5E74FFFFFEFDFC9000CCE0B9
:105D5A00F8A3E0F9A3E0FAA3E0FBC3121EBB603884
:105D6A007F807E967D187C4B9000CCE0F8A3E0F90A
:105D7A00A3E0FAA3E0FB121A4A6002501B7F807E5E
:105D8A00967D187CCB9000CCE0F8A3E0F9A3E0FA6A
:105D9A00A3E0FB121A4A500F9000CCE0FCA3E0FDEE
:105DAA00A3E0FEA3E0FF229000CCE0FCA3E0FDA369
:105DBA00E0FEA3E0FF121B069000D0121F5E9000C7
:105DCA00D0E0FCA3E0FDA3E0FEA3E0FFEC121AC8BA
:105DDA00C8ECC8C9EDC9CAEECACBEFCB9000CCE07B
:105DEA00FCA3E0FDA3E0FEA3E0FF1217AFE4FBFA79
:105DFA00F9F8121A4A602640249000D0E0FCA3E089
:105E0A00FDA3E0FEA3E0FFEF24FFFFEE34FFFEED6B
:105E1A0034FFFDEC34FFFC9000D0121F5E9000D0DE
:105E2A00E0FCA3E0FDA3E0FEA3E0FFEC121AC82207
:101B3D00E9D2E7C933E833F892D5EDD2E7CD33ECEE
:071B4D0033FC5002B2D52267
:101B5400EC30E7100FBF000C0EBE00080DBD0004F2
:101B64000BEB6014A2D5EB13FCED92E7FD2274FF9E
:101B7400FCFDFEFF22E480F8A2D574FF13FC7D80F7
:031B8400E480EF0B
:101B8700F920E73624F950037907E4F42402FBE54A
:101B970082158270021583DBF6E024FB501BE96097
:101BA70014E4F0E582158270021583E004F0B40AAC
:0D1BB70008E4F0D9EE7401F00A22C2D52234
:101BC400ED33EC3392D5FA602AB4FF33EDC2E77BF0
:101BD400FF60067A1B79E9E4227A1B79F220D504A6
:101BE4007A1B79ED224E614E002B494E46002D4959
:101BF4004E4600E47A08F0A3DAFC7B00740722C0A6
:101C040083C082ECC0E0EDC0E0EEC0E0EFC0E0EAEB
:101C140075F010A4CAABF075F04DA42BFBE435F0BD
:101C2400FCEA2410FAEB34C5FBEC34D9FCEDC2E732
:101C3400FF75F056A4F42411C5F0F434C58FF0A454
:101C44002AE5F03BE43CF020E714121D46D0E0FF07
:101C5400D0E0FED0E0FDD0E0FC1219AD8014F40415
:101C6400121D46D0E0FFD0E0FED0E0FDD0E0FC1233
:101C740018A4D082D083E0FAEDD2E7CD33EC33243C
:101C840082FBE4C3CF33CFCE33CECD33CD33DBF3BE
:101C94007B0775F00A846004F0A31B0AE5F0F0A347
:101CA4008FF0740AA4FFACF08EF0740AA42CFEAC7E
:101CB400F050010C8DF0740AA42CFDE435F0F0A36F
:051CC400DBDE740722C5
:101CC900C0E0EFFBEEFAEDF9ECF81218A4D0E0F55C
:101CD900F0EFFBEEFAEDF9ECF8121F12A3A3A3A3A0
:101CE900E8C0E0E9C0E0EAC0E0EBC0E0C0F01218EB
:101CF900A4121F2EA3A3A3A31217B3D0F0D0E0FB05
:0D1D0900D0E0FAD0E0F9D0E0F8D5F0D42217
:101D16003F8000004120000042C80000447A0000D5
:101D2600461C400047C35000497424004B18968057
:101D36004CBEBC205A0E1BCA6753C21C749DC5AE4E
:101D4600FB60065407601C2323121D74EB54386095
:101D560009121D60121D6F1218A4ECF8EDF9EEFAC7
:101D6600EFCB22EB121D6F80F1543803241C901D1B
:101D760016FE93FC0EEE93FD0EEE930ECE93FF220F
:10656F0002217BE493A3F8E493A34003F68001F2A6
:10657F0008DFF48029E493A3F85407240CC8C3332D
:10658F00C4540F4420C8834004F456800146F6DFFC
:10659F00E4800B0102040810204080906886E47E9E
:1065AF00019360BCA3FF543F30E509541FFEE493F1
:1065BF00A360010ECF54C025E060A840B8E493A3B8
:1065CF00FAE493A3F8E493A3C8C582C8CAC583CAE3
:1065DF00F0A3C8C582C8CAC583CADFE9DEE780BE9B
:0168C60000D1
:101D8600C2D530F707B2D563F0FF05F030E70CB2E5
:101D9600D5F4048463F0FF05F080018430D502F4A5
:021DA600042215
:101DA800BB010689828A83E0225002E722BBFE0239
:091DB800E32289828A83E493226C
:101DC100BB010CE58229F582E5833AF583E02250D7
:101DD10006E92582F8E622BBFE06E92582F8E22221
:0D1DE100E58229F582E5833AF583E493223B
:101DEE00BB010689828A83F0225002F722BBFE01D4
:021DFE00F322CE
:101E0000EF8DF0A4A8F0CF8CF0A428CE8DF0A42EF6
:021E1000FE22B0
:101E1200C2D5EC30E709B2D5E4C39DFDE49CFCEEEB
:101E220030E715B2D5E4C39FFFE49EFE12200EC335
:101E3200E49DFDE49CFC800312200E30D507C3E430
:061E42009FFFE49EFE225A
:101E4800C5F0F8A3E028F0C5F0F8E5821582700225
:061E58001583E038F022C2
:101E5E00E88FF0A4CC8BF0A42CFCE98EF0A42CFC23
:101E6E008AF0EDA42CFCEA8EF0A4CDA8F08BF0A4A1
:101E7E002DCC3825F0FDE98FF0A42CCD35F0FCEB00
:101E8E008EF0A4FEA9F0EB8FF0A4CFC5F02ECD39C5
:0F1E9E00FEE43CFCEAA42DCE35F0FDE43CFC2232
:10680000C2D5E830E70FB2D5E4C39BFBE49AFAE4C3
:1068100099F9E498F8EC30E717B2D51268361220EF
:106820009FE4C39BFBE49AFAE499F9E498F88003A7
:1068300012209F30D50DE4C39FFFE49EFEE49DFD32
:04684000E49CFC22B6
:0E1EAD00C3E49FFFE49EFEE49DFDE49CFC2246
:101EBB00EB9FF5F0EA9E42F0E99D42F0E89C45F07D
:011ECB0022F4
:101ECC00BB010789828A83021F065005E9F80221AB
:101EDC0031BBFE05E9F802213D89828A83021F127B
:101EEC00BB010789828A83021F5E5005E9F8022133
:0A1EFC0063BBFE05E9F802216F2226
:0C1F0600E0FCA3E0FDA3E0FEA3E0FF224E
:101F1200E493FC740193FD740293FE740393FF2215
:0C1F2200E0F8A3E0F9A3E0FAA3E0FB2242
:101F2E00E493F8740193F9740293FA740393FB2209
:101F3E00BB010789828A83021F225005E9F802211C
:101F4E0049BBFE05E9F802215689828A83021F2EBB
:0C1F5E00ECF0A3EDF0A3EEF0A3EFF022F6
:101F6A00A8828583F0D083D082121F81121F81122A
:101F7A001F81121F81E473E493A3C583C5F0C5834F
:101F8A00C8C582C8F0A3C583C5F0C583C8C582C8C1
:011F9A002224
:101F9B00F8E0FBA3A3E0F925F0F0E58215827002CF
:071FAB001583E0FA38F02273
:091FB200EBF0A3EAF0A3E9F02230
:101FBB00D083D082F8E4937012740193700DA3A3B5
:101FCB0093F8740193F5828883E4737402936860C9
:061FDB00EFA3A3A380DFC9
:101FE100D083D082F8E4937012740193700DA3A38F
:101FF10093F8740193F5828883E473740293B5F0C6
:0D200100067403936860E9A3A3A3A380D82D
:10692700EFB40A07740D126932740A309811A899E6
:10693700B8130CC2983098FDA899C298B811F630D0
:0769470099FDC299F59922A8
:10000E00C3EE6480948040028007C3E49FFFE49EA9
:02001E00FE22C0
:10200E00BC000BBE0029EF8DF084FFADF022E4CCB6
:10201E00F875F008EF2FFFEE33FEEC33FCEE9DEC7F
:10202E00984005FCEE9DFE0FD5F0E9E4CEFD22EDC5
:10203E00F8F5F0EE8420D21CFEADF075F008EF2F0F
:10204E00FFED33FD4007985006D5F0F222C398FD00
:05205E000FD5F0EA229D
:1020630075F008758200EF2FFFEE33FECD33CDCC34
:1020730033CCC58233C5829BED9AEC99E5829840B7
:102083000CF582EE9BFEED9AFDEC99FC0FD5F0D694
:10209300E4CEFBE4CDFAE4CCF9A88222B800C1B9BE
:1020A3000059BA002DEC8BF084CFCECDFCE5F0CBFC
:1020B300F97818EF2FFFEE33FEED33FDEC33FCEB35
:1020C30033FB10D703994004EB99FB0FD8E5E4F9F0
:1020D300FA227818EF2FFFEE33FEED33FDEC33FCDD
:1020E300C933C910D7059BE99A4007EC9BFCE99AD1
:1020F300F90FD8E0E4C9FAE4CCFB2275F010EF2F16
:10210300FFEE33FEED33FDCC33CCC833C810D70715
:102113009BEC9AE899400AED9BFDEC9AFCE899F850
:0E2123000FD5F0DAE4CDFBE4CCFAE4C8F922E3
:0C213100E6FC08E6FD08E6FE08E6FF22DA
:0C213D00E2FC08E2FD08E2FE08E2FF22DE
:0D214900E6FB08E6F908E6FA08E6CBF82206
:0D215600E2FB08E2F908E2FA08E2CBF82209
:0C216300ECF608EDF608EEF608EFF622A8
:0C216F00ECF208EDF208EEF208EFF222AC
:00000001FF
